:10747800758400852ED2852FD3E4F52FF52E30386C
:1074880010E50D852DF0A4252EF52EE5F0352FF508
:107498002F229074B4303E031274A422E50E251BEB
:1074A800F50EE51F351AF51F93F50D227F828588A5
:1074B8008C8F9295989B9EA1A4A7AAADB0B3B6B99C
:1074C800BBBEC1C3C6C9CBCED0D3D5D7D9DCDEE0CD
:1074D800E2E4E6E7E9EBEDEEF0F1F2F4F5F6F7F8C1
:1074E800F9FAFBFCFCFDFDFEFEFEFEFEFEFEFEFEC6
:1074F800FEFDFDFCFCFBFAFAF9F8F7F6F4F3F2F0FE
:10750800EFEDECEAE8E7E5E3E1DFDDDBD8D6D4D15F
:10751800CFCDCAC8C5C2C0BDBAB7B4B2AFACA9A6B0
:10752800A3A09D9A9794908D8A8784817E7A777498
:10753800716E6B6865625F5C595653504D4A47449B
:10754800423F3C393734322F2D2A282624211F1D4B
:107558001B1918161412110F0E0C0B0A0807060532
:107568000404030202010100000000000000000002
:107578000001010202030405060708090A0B0D0EA3
:107588001011131516181A1C1E20222427292B2E19
:10759800303335383A3D404245484B4E51545659A0
:0C75A8005C606366696C6F7275787B7FB5
:107CA900D2F4C2F5C2F675840F85F0C81279F5745D
:107CB90003127CF81279E57403127CF81279D41254
:107CC90079D47403127CF81279D47402127CF812F4
:107CD90079D47428127D647406127D64740E127D41
:107CE900647401127D641279E57480127D6422C086
:107CF90000A2E092F3A2E192F2A2E292F1A2E3924F
:107D0900F0D2F475840F85F0C8C2F47830D8FE85B6
:107D1900F0C87830D8FED00022C00075840FA2E4E4
:107D290092F3A2E592F2A2E692F1A2E792F0D2F4DE
:107D390085F0C8C2F47830D8FE85F0C87830D8FE0E
:107D4900D00022EF75840FD2F5C2F685F0C8127DF6
:107D5900221279D4127CF81279D42275840FC2F5D3
:107D6900C2F685F0C8127D221279D4127CF81279F4
:107D7900D422EF14A2E492E6C2E4D2E7127D64228F
:107D8900740F127D6422740D127D64227F01127DAD
:107D99007B78107F20127D4CD8F9227F11127D7BD0
:0A7DA90078107F20127D4CD8F922DB
:10733B00C293758400D2C2C2C6D2C6C2C4D2C5C261
:10734B00C330C3FD74A0F5C2C2C5C2C330C3FD8E2A
:10735B00C2C2C330C3FD8FC2C2C330C3FD8DC2C214
:10736B00C330C3FDD2C4C2C320C4FD1279E5D2938E
:10737B0022758400C2C3D2C530C3FD74A0F5C2C24E
:10738B00C5C2C330C3FD8EC2C2C330C3FD8FC2C2E0
:10739B00C330C3FDC2C4D2C5C2C330C3FD74A1F593
:1073AB00C2C2C5C2C330C3FDC2C2C2C330C3FD8596
:1073BB00C207D2C4C2C320C4FD22D2C2C2C6D2C627
:1073CB00D2C4C2C320C4FD22C293758400D2C2C2F0
:1073DB00C6D2C6C2C4D2C5C2C330C3FD74A0F5C2E7
:1073EB00C2C5C2C330C3FD8EC2C2C330C3FD8FC280
:1073FB00C2C330C3FD8C838D827B80E0A3F5C2C2F8
:10740B00C330C3FDDBF5D2C4C2C320C4FD1279E582
:10741B00D29322758400C2C3D2C530C3FD74A0F5CC
:10742B00C2C2C5C2C330C3FD8EC2C2C330C3FD8F3F
:10743B00C2C2C330C3FDC2C4D2C5C2C330C3FD7404
:10744B00A1F5C2C2C5C2C330C3FD8C838D82C2C33A
:10745B0030C3FDE5C2F0A31BBB01F3C2C2C2C330F4
:0D746B00C3FDE5C2F0D2C4C2C320C4FD229F
:030003000259900F
:01000B0032C2
:030013000276EF83
:1065E60075FF0775FFDE75FFAD75840F75E10775DD
:1065F600E21475E34475840F75A43575A50975A66F
:10660600BB75A7FF759CFF759D00759EF0759FF87D
:1066160075D8FF75E8FF75F80F75AD0F75840175B0
:10662600893075888F75840275893075888F758471
:106636000F758A80758C67780874FF00000000006B
:1066460000000000000000D5E0F1D8EDE58C30E751
:10665600FB759701758A0043890475840075B71028
:1066660075840F438901758D02758F01758E0474CB
:1066760080D5E0FD438902E58930E4FB7597027514
:10668600840075D10775840075BB0175BA0075BCA9
:10669600F075C70075C60075C5FF75C4FF75E800BF
:1066A60075840275BB0475BA0075BCF175C60075B4
:1066B600C4FF75E88075840075D48475840175D42B
:1066C60084758400C2F8759A47759D1A75F8017528
:1066D600870075840075B90075A9007591007598D5
:1066E6005075840175989075840075C04075C30017
:1066F60075CFC9758400758E1075892175880575E5
:106706008400758A00758BE0758CF4758DE043887E
:106716004075840075C90075CA0075CB0075CC003C
:1067260075CD0075840175C91875CA8075CBFB7562
:10673600CDFB75CC80D2CA75840275C91875CAA6F8
:1067460075CBAF75CDAF75CCA6D2CA75840075EF83
:106756000275A8AC75B83D75E6B075E71D75F6000F
:1067660075F741789D760A769E780A789F76067543
:07677600A8959000007F00D0
:10677D007E20E4F0A3DFFCDEFA789D760A789E7623
:0E678D000A789F7606D29375E8FF1273C52234
:10794E0075840FD2FD2275840FC2FD22E490FC00D7
:10795E00732275840FD2EA2275840FC2EA227584CF
:10796E000FA2EC2275840FD2FC2275840FC2FC226A
:10797E0075840FC2FF2275840FD2FF2275840FA269
:10798E00FA2275840FA2F92275840FA2DD22A2922B
:10799E002275840FA2DA2275840FA2DB2275840F62
:1079AE00A2D82275840FA2D9220000000000000088
:1079BE0000000000000000000000000000000000B9
:1079CE00000000000022C000C001790878B4D8FE83
:1079DE00D9FAD001D00022C000C0E078997605E631
:1079EE0070FDD0E0D00022C000C0E07899760FE69E
:1079FE0070FDD0E0D00022C000C0E078997664E639
:107A0E0070FDD0E0D00022EF75F064842430900039
:107A1E0054F0E5F0A375F00A842430F0A3E5F024C9
:107A2E0030F022EF75F064842430900054F0E5F0CD
:097A3E00A375F00A842430F0A3C2
:107A4700E5F02430F0900054E0B4300B7420F0A33C
:107A5700E0B430037420F02275F06484F6E5F00892
:107A670075F00A84F608A6F0082285060722228503
:037A7700050622DF
:101A1A00C0D0C000C001C083C082C0E0C0F0C0070F
:101A2A00A291304F01B37825E233F208E233F2088B
:101A3A00E233F208E233F208E233F208E233F20860
:101A4A00E233F208E233F208E233F208E233F20850
:101A5A00E233F208E233F208E233F208E233F20840
:101A6A00E233F208E233F208E233F208E233F20830
:101A7A00E233F208E233F208E233F208E233F20820
:101A8A00E233F208E233F208E233F208E233F20810
:101A9A00E233F208E233F208E233F208E233F20800
:101AAA00E233F208E233F208E233F208E233F208F0
:011ABA00E249
:101ABB0033F208E233F208E233F208E233F208E2DF
:101ACB0033F208E233F2305B35901EE4784CE218C7
:101ADB00203C03936028E218937023E21893601E56
:101AEB00E218937019E218936014E21893600FE2F6
:101AFB001893700AE218937005E218936003021CA6
:101B0B00C0754000E2189313924750037540387527
:101B1B002200E21893139214500363401CE21893B3
:101B2B00139213500363400EE21893139212500357
:101B3B00634046E218931392115003634023E2185B
:101B4B00931392108522415003634051752200E29A
:101B5B0018931392145003634068E2189313921373
:101B6B005003634075E21893139212500363407A4B
:101B7B00E21893139211500363403DE218931392B2
:101B8B0010852242500363401F752200E218931305
:101B9B009217500363404FE218931392165003634E
:101BAB004026E218931392155003634052E21893A8
:101BBB001392145003634029E218931392135003AA
:101BCB00634015E21893139212500363400BE21813
:101BDB00931392115003634045E2189313921085AF
:101BEB0022435003634062E2189313921450036331
:101BFB004031E218931392135003634019E2189388
:101C0B00139212500363400DE21893139211500379
:101C1B00634007E2189313921085224450036340EC
:101C2B0043752200E21893139216E2189313921540
:101C3B00E21893139214E21893139213E21893136E
:101C4B009212E21893139211E218931392108522B9
:101C5B0045C24CE54565406035D24C23F8902435A0
:101C6B0093F9902434E8936025B40104B247801EA5
:0E1C7B00B40205E862418016B40305E8624237
:101C8900800EB40405E862438006B4052AE862447C
:101C9900A247924890004DE541F090004EE542F090
:101CA90090004FE543F0900050E544F0304B06D2E8
:101CB9004AC24B8002D24B121CD4D007D0F0D0E0DC
:101CC900D082D083D001D000D0D022C0D0C000C0F3
:101CD900E0303F4EE552B40833A242B392B3787D67
:101CE900E66036167882E6A2E7304401B392429262
:101CF900B2A2E7787EE633F6787FE633F67880E6B7
:101D090033F67881E633F67882E633F6D5520375F1
:101D19005208D0E0D000D0D022C257D0E0D000D0B5
:101D2900D022D0E0D000D0D022C0D0C000C001C0A5
:101D390083C082C0E0C0F0A291204E01B3780DE2C9
:101D490013F208E213F208E213F208E213F208E2CE
:101D590013F208E213F208E213F208E213F208E2BE
:0D1D690013F208E213F208E213F208E2138D
:101D7600F208E213F208E213F208E213F208E213A1
:101D8600F208E213F208E213F208E213F208E21391
:101D9600F208E213F208E213F208E213F2901EE4EC
:101DA600780DE2089313920FE2089313920EE2085D
:101DB6009313920DE2089313920CE2089313920B7D
:101DC600E2089313920AE20893139209E208931326
:101DD6009208852146E2089313920FE20893139224
:101DE6000EE2089313920DE2089313920CE2089305
:101DF60013920BE2089313920AE20893139209E2F4
:101E06000893139208852147E2089313920FE2087C
:101E16009313920EE2089313920DE2089313920C19
:011E2600E2D9
:101E2700089313920BE2089313920AE20893139212
:101E370009C208852148305B3DE546902234854735
:101E470021300E02058393602D14F875F003A490DA
:101E570020E52582F582E5F03583F583E493F9A340
:101E6700E493901FE4654893C965479329B401003B
:101E770050048834D241121E8FD0F0D0E0D082D0E7
:101E870083D001D000D0D022303D24788316E6706D
:101E97001E76087886E6A2E1304501B392B2A2E148
:101EA7007884E613F67885E613F67886E613F62245
:101EB700EF9020E475F003A42582F582E58335F0E1
:101EC700F583C23D7400937884F67401937885F6A0
:101ED7007402937886F6C23FC23ED23D22000000CC
:101EE70000000000000000000000000000000000EB
:101EF70000000000000000000000000001000000DA
:101F070000000000000000000000000001000000C9
:101F170000000000010000000100010101000000B5
:101F270000000000000000000000000001000000A9
:101F37000000000001000000010001010100000095
:101F47000000000001000000010001010100000085
:101F5700010001010100010101010101010000006F
:101F67000000000000000000000000000100000069
:101F77000000000001000000010001010100000055
:101F87000000000001000000010001010100000045
:101F9700010001010100010101010101010000002F
:101FA7000000000001000000010001010100000025
:101FB700010001010100010101010101010000000F
:101FC70001000101010001010101010101000101FD
:101FD70001010101010101010101010101000101EB
:101FE70002010202030102020302030304010202C7
:101FF70003020303040203030303030405010202AC
:102007000302030304020303040304040502030396
:10201700040304040503040404040505060102027D
:102027000302030304020303030304040502030377
:10203700040303040503040405040505060203035A
:102047000403040405030404050405050603040446
:10205700050405050604050506050606070102022F
:102067000302030304020303040304040502030336
:102077000403040405030404050405050602030319
:102087000403040405030404050405050603040406
:1020970005040505060405050605060607020303EC
:1020A70004030404050304040504050506030404E6
:1020B70005040505060405050605060607030404C9
:1020C70005040505060405050605060607040505B6
:1020D70006050606070506060706070708FDD00CCE
:1020E70073700E3CF01AAF101E7F9022EC7026D64C
:1020F700F02ACBB02CA3F032BEB03417D03CB6D008
:10210700461FB04E77F050F950526AB056DE9058DD
:10211700BA306ACF3072D270745CD076E8F0786BE0
:10212700D098E5709AF8309CBB50A40F70AA7A70CB
:10213700B26730B45DB0B8FCB0C26F50C655D0CAF4
:102147003D90D489B0DA94F0DCD790E463B0EA0B21
:10215700F0F43170F8DD310AB571148FF118D1D16F
:1021670026EB512AF6112C8B71463F5148B1F14AA3
:10217700ACB14CC4F152D9B1546D915A2EF162BD34
:10218700116687916A9AD16CF29172D5517819F1DB
:0D2197008C71B192D8D19A32D1AA47D1B241
:1021A4005A91B452F1C67531CC1D71D2A951DCD00B
:1021B400B1E85E11EA2B11F2EED212F392147D32E1
:1021C40016973226D8B232C5F234F7124AEA524C84
:1021D4009F5254A5D2582B725A7552644FD268C17B
:1021E400726ADC326C78D2865F128C83729C4EB237
:1021F400A66972AC1C72B433D2CC18F2EABB330CAD
:10220400CE33141EB32803F32EE51332F853349857
:10221400735848F36472736845738617B3947313E1
:10222400A63C93B221D3B41B53B829B3C641F3D807
:10223400000000000000000000000000000000009A
:10224400000000000000006A000000000000620DB1
:102254000000000000000000006F004800000000C3
:102264000000000000000000000000006C220000DC
:1022740000000000000000000000000000005B00FF
:10228400000000000000000000004100001E47594B
:10229400000000260000001D0000100000350000B2
:1022A400003D006B0043000000000000004B0005EF
:1022B40000000000000000380023000000000000BF
:1022C400000000000000004C0000000000000000BE
:1022D40000000000000000000000000032000004C4
:1022E40000000000000000000000126000370A0037
:1022F400000000000000000000000008000061135E
:1023040046000000000000254D340000572911004C
:102314000000000000640000000000000000000055
:1023240000003A4A00002E4F190000001F00000070
:102334000000006300000000000000270000001BF4
:10234400000000000000000B5F3C006E5D440000D4
:10235400006D000000000000000000530000360083
:1023640000283F5E00000000000000000300003071
:102374000070000000690040670000000000005584
:1023840000004200002100000000000015000000D1
:102394000000000000000000005C001700000020A6
:1023A400000068020054000E58001C0000000000E9
:1023B4000000005A000000000000002F0000002B65
:1023C40000000000240000006600390000000051F5
:1023D4000000000900520000004500000000000059
:1023E40000310000002A0C000000001A0000000068
:1023F40000560000334E0000000000000000000002
:10240400002C1400003B07003E0000000000000008
:1024140000000000001800001600502D06004900BE
:102424000000000000000000650F00000001000033
:10243400000000000000060000000600060005027F
:10244400060006000600040406000504020806004F
:102454000000060006000600060004080600060048
:102464000600050806000600021006000600030127
:1024740000000600060002020600060004400600F2
:10248400060004100600060006000600060006000A
:1024940006000510060006000600060006000600F9
:1024A40001010600060006000600030206000600FD
:1024B40000000600060005010600040202040600EE
:1024C400060006000600060006000600060004805A
:1024D40006000201042006000600060006000600AD
:1024E40006000600060006000600060006000600B8
:1024F40006000600040106000600060006000600A9
:10250400031006000600060006000600060006008A
:0D251400060006000600060006000308068B
:102521000006000600060003040600060006000679
:03253100000600A1
:10599000758400C2CA85CC3885CD3775CC0075CDED
:1059A00000D2CA10CF02D25A32305A0BC25AE5374F
:1059B000C394364002800122788E798C7B06E7F60C
:1059C0001819DBFAA63718A638AA38AB37AE02AFDB
:1059D00003EEC4035407FEEFC403FF54F84EFEEF7A
:1059E0005407FF78037989C3E79AFC09E79BFD090F
:1059F00050066304FF6305FFC3EC9EED9F5074D80F
:105A0000E6789679947C06E7F61819DCFAA603186E
:105A1000A6027991AE02AF03EEC423541FFEEFC479
:105A200023FF54E04EFEEF541FFF7803C3E79AFCB8
:105A300009E79BFD0950066304FF6305FFC3EC9E65
:105A4000ED9F502FD8E6788F7A007B007C00790498
:105A5000EA26FA08EB36FB08EC3400FCD9F2EC132A
:0D5A6000FCEB13FBEA13FAEC13EB13F53625
:105A6D00EA13F535D23A22303A31C23A125AA950D8
:105A7D002A853C3D853B3C853A3B85393A8507393E
:105A8D00303913E53F6F600EE507B53A0EB53B0BA8
:105A9D00B53C08B53D0585073ED23B22905BC4E57C
:105AAD003693FF905AF023232582F582E583340047
:105ABD00F583125ACF400A0F125ACF40040F125AD3
:105ACD00CF22E493F9A3E493FAA3E493FBA3E49325
:105ADD00FCA3C3E5359AE536995007C3EC9535EB34
:105AED00953622EA25DD89DD89D324D324CBD2CB8B
:105AFD00D2C4DBC4DBBE39BE39B7CAB7CAB18EB1A9
:105B0D008EAB87AB87A59CA59CA000A0009A969A0A
:105B1D009695D895D891E591E58D858D8588AF8839
:105B2D00AF840C840C7F9A7F9A7B497B49771B77D6
:105B3D001B730F730F6F276F276B576B5767AB6710
:105B4D00AB642C642C60C660C65D795D795AFE5AD3
:105B5D00FE5970597057E257E25661566154E75439
:105B6D00E7537453745207520750A050A04F404F43
:105B7D00404DE64DE64C934C934B414B4149F54915
:105B8D00F548B548B547764776463E463E45084505
:105B9D0008432A432A40E440E43F533F533E3E3EF0
:105BAD003E3C943C943A863A8639183918380500AB
:105BBD000000000000000032323232323232323216
:105BCD0032323232323232323232323232323232A8
:105BDD003232323232323232323232323232323298
:105BED003232323232323232323232323232323288
:105BFD00313130302F2E2D2D2D2C2C2B2A292928CB
:105C0D0027262525242323222120201F1E1E1D1C6F
:105C1D001C1B1A1A1A1A19191918181817171717E9
:105C2D00161616161515151514141414131313131F
:105C3D00121212121111111110101010100F0F0F4E
:105C4D000F0F0E0E0E0E0D0D0D0D0C0C0C0C0B0B77
:105C5D000B0B0B0B0A0A0A0A0A090909090909089B
:105C6D0008080808080707070707070606060606B7
:105C7D0006060505050505050404040404040403CE
:105C8D0003030303030302020202020202010101E4
:105C9D0001010101010101010101010000000000EC
:105CAD0000000000000000000000000000000000E7
:075CBD0000000000000000E0
:10709900C007C0007F01127D7B7F4C127D4C7F545D
:1070A900127D4C7F52127D4C7F20127D4C2048046A
:1070B9007F3080027F31127D4C7F20127D4C900001
:1070C9004EE0784B127A67784B8607430730127D7A
:1070D9004C088607430730127D4C750720127D4CFA
:1070E90090004FE0784B127A5F784B860743073060
:1070F900127D4C088607430730127D4C08860743EA
:107109000730127D4C750720127D4C90004DE078B8
:107119004B127A67784B8607430730127D4C0886F5
:1071290007430730127D4C750720127D4CD000D0E3
:107139000722C007C0007F11127D7B7F4C127D4C56
:10714900750720127D4C204D047F3080027F31125B
:107159007D4C7F20127D4C90015BE0784B127A6761
:10716900784B8607430730127D4C08860743073062
:10717900127D4C750720127D4C90015CE0784B1212
:107189007A5F784B8607430730127D4C08860743A0
:107199000730127D4C088607430730127D4C75076E
:1071A90020127D4C90015DE0784B127A67784B860E
:1071B90007430730127D4C088607430730127D4C80
:1071C900750720127D4C90015EE0784B127A677842
:1071D9004B8607430730127D4C0886074307301258
:0771E9007D4CD000D007220D
:106DDB00003800512372461765340E5F2D7C48191D
:106DEB006B3A1C4D3F6E5A0B792812433160540598
:106DFB007726001F3D227A654758756A48570F1052
:106E0B00322D6877554A120D2F301D02203F6778BF
:106E1B005A45006245270B694E2C157750321E7C64
:106E2B005B39294B6C0E224067053C5E791B37554D
:106E3B00721052301775593B1C7E472502604C2E41
:106E4B00096B7B193E5C701235576E0C2B4965072D
:106E5B002042264463012D4F680A33517614385A69
:106E6B007D1F0F6D4A28046641231A785F3D11730D
:106E7B005436741631537F1D3A58610324466A0801
:106E8B002F4D5D3F187A56341371482A0D6F4321ED
:106E9B0006644F2D0A68442601635A381F7D51330F
:106EAB001476660423416D0F284A73113654781AF1
:106EBB003D5F1D7F583A16745331086A4D2F03619D
:106ECB004624345671133F5D7A18214364062A48D1
:106EDB006F0D690B2C4E620027457C1E395B7715B5
:106EEB003250402205674B290E6C553710725E3CB1
:106EFB001B793B597E1C305275172E4C6B0925475D
:106F0B00600212705735197B5C3E076542200C6E90
:106F1B00492B004307440D4E0A49195A1E5D14575D
:106F2B001350317236753C7F3B78286B2F6C25667E
:026F3B002261D1
:10853800788276ACA24DE433FFC4333354C0FE9046
:10854800015DE0FD541F25E04EFE90015BE0FC5408
:1085580010C4540F4E7881F6EC540FC454F0FE90BA
:10856800015CE0FC54F0C4540F4E7880F6EC540FD4
:10857800C454F0FE90015EE0FC541EC3134E787F95
:10858800F6EF3395E0FE74DB2FF582746D3EF583CC
:10859800E493FFED906DDD93FEEF6EFF90015BE0DD
:1085A800906DFD936FFF90015CE0906E1D936FFFDF
:1085B800EC906F1D936F787EF690015EE030E004DA
:0B85C800E64480F6D257787D7628222A
:1090F600758401309914C29920500F900159E0707F
:1091060009D250D29C789776042230983790015A2B
:10911600E06401702DE54975F0058420551124EFB2
:10912600F582E43400F583E599F0C298D2552224FD
:1091360004F582E43401F583E599F0C298C255D26C
:059146005622C2982230
:1080AB00758401209803028171205213209A0DE5EB
:1080BB00997009D252D253754A0AF549C298229047
:1080CB00015AE0FF6401702CE54975F005842055D9
:1080DB001024EFF582E43400F583E599F0D2558056
:1080EB00102404F582E43401F583E599F0C255D2EE
:1080FB0056C29822EFB4021AAB530555E555AA5454
:10810B007002055414F9E5991284D890015A74033E
:10811B00802090015AE0FFB4031CAB530555E55585
:10812B00AA547002055414F9E5991284D890015A97
:10813B007404F0C29822EFB4042990018CE0FF0480
:10814B00F074632FF582E43401F583E599F0C2985E
:10815B0090018CE0B4281C90018E7401F0E4900126
:10816B005AF022C2982230990AC299900159E070B4
:04817B0002C25522C5
:1098C10020512212798443E740754A0AE4F5499010
:1098D1000159F090015AF0C250D251758401759826
:0698E10090C29CF59922E3
:108ECC0090018DE0705C9001ABE0FF7025D39001B8
:108EDC0060E0948690015FE094674008E4F0A3742E
:108EEC0002F0800E900160E02428F090015FE034E5
:108EFC0000F0900160E02FFF90015FE03400FE1263
:108F0C00737C9001ABE02463F582E43401F583EFCC
:108F1C00F09001ABE004F0E0B42807E4F090018D90
:038F2C0004F0222C
:108A3F0090018EE0607A900161E0FEA3E0FFC394A5
:108A4F0002EE94005006E490018EF0229001ABE00C
:108A5F007C002FFFEC3EFE12737C9001ABE0246391
:108A6F00F582E43401F583E0FD6F60179001ABE010
:108A7F00FF900162E02FFF900161E03400FE12735E
:108A8F003BD2549001ABE004F0E0B42823E4900112
:108A9F008EF09001ABF0900161E07004A3E06402EE
:108AAF00700E30540BC2541286FE128F8F128FEB42
:018ABF002294
:108D97003050647584019001A0E0B40D00505590E7
:108DA7008DADF8282873028DD4028DD7028DDA0293
:108DB7008DDD028DE0028DE3028DE6028DE9028DE5
:108DC700EC028DEF028DF2028DF5028DF802980EFE
:108DD700029A230293AE0295B10298E702005E025F
:108DE70097DB0297080295ED0293F10299C2029868
:088DF700690299A71299DC2220
:10980E007897E67028759898754A0AF54990005B26
:10981E00E0B401079001A07404F022E490015AF024
:0E982E00900159F09001A0E004F012797E2222
:109A230090015A7401F0E4900159F0C2559001A0DD
:049A3300E004F02239
:1093AE0090005BE01475F005A4B54919E4B5F0150D
:1093BE00759898127984E4900159F090015AF090C2
:1093CE0001A07404F0E54975F00584AFF0BF0112F9
:1093DE00C256E4900159F090015A04F09001A0E0B9
:0393EE0004F02266
:1095B100E54975F00584AFF0BF043020561EE5493A
:1095C10075F00584FF24EFF582E43400F583E4F0BF
:1095D10074042FF582E43401F583E4F0E490015939
:0C95E100F090015AF09001A0E014F0227C
:1098E70090005BE075F005A424FDB5491590005282
:1098F700E0F599E4900159F090015AF09001A0E049
:0399070004F02247
:0D005E00900053E0F5999001A0E004F0221D
:1097DB0090005BE0FD75F005A4FFE549B50723E4B8
:1097EB00B5F01FEDB414079001A07409F0221279A3
:1097FB007EE4900159F0C25590015AF09001A0E01F
:03980B0004F02244
:10970800E549B46412127984E4900159F090015A41
:10971800F09001A07409F0E54975F00584AFF0BF39
:109728000112C256E4900159F090015A04F09001D8
:05973800A0E004F02296
:1095ED00E54975F00584AFF0BF043020561EE549FE
:1095FD0075F00584FF24EFF582E43400F583E4F083
:10960D0074042FF582E43401F583E4F0E4900159FC
:0C961D00F090015AF09001A0E014F0223F
:1093F100E5496465703C90018DE0B4012F7553011E
:1094010075540175555FE4900159F090015AF0755A
:109411008401AB530555E555AA547002055414F95E
:10942100128492F5999001A0E004F0229001A074B9
:039431000CF0221A
:1099C200758401AB53AA54A955128492F599E49077
:0A99D200018BF09001A0E004F022E8
:1098690075840190018BE0FF04F074632FF582E4A5
:109879003401F583E0F59990018BE0D39428400BEE
:0C988900E490018DF09001A0E004F022BA
:1099A700E549B46915C250C251E49000EDF0900149
:0B99B70059F090015AF09001A0F0223E
:1099DC00C250C251E4F5499000EDF0900159F0905D
:0899EC00015AF09001A0F022E5
:1090A0003052527584019001A1E0B40A00504390FF
:1090B00090B6F82828730290D40290D70290DA0272
:1090C00090DD0290E00290E30290E60290E90290C7
:1090D000EC0290EF0296D202962902966202996AF9
:1090E000029A930298950294B902969A02990A02FA
:0690F0009A82129AA322ED
:1096D200E549703175989890005BE0B401131279F6
:1096E20084E490015AF0900159F09001A17403F0C2
:1096F2002212797EC255E490015AF0900159F090FD
:0697020001A1E004F022C9
:1096290090005BE01475F005A4B54911E4B5F00D9F
:109639007598981279849001A17403F022E549750F
:10964900F00584AFF0BF0110C256C25590015A749B
:0996590001F09001A1E004F022EF
:10966200E54975F00584AFF0BF042C20561EE5498C
:1096720075F00584FF24EFF582E43400F583E4F00D
:1096820074042FF582E43401F583E4F0E490015A86
:08969200F09001A1E014F022A8
:10996A0090005BE075F005A424FDB54911758401EA
:0F997A00900052E0F599C2559001A1E004F0224F
:109A9300758401900053E0F5999001A1E004F02250
:1098950090005BE0FFB414079001A17406F022EF7D
:1098A50075F005A4B54914E4B5F01012797E900160
:0C98B500A1E004F0C255E490015AF0223A
:1094B900E54975F00584AFF0BF0111C256C2559058
:1094C900015A7401F09001A1E004F022E549B46465
:1094D9001F12797E90018EE0700B90015AF0900175
:1094E900A17408F022E490015AF09001A17409F0E6
:0194F9002250
:10969A00E54975F00584AFF0BF042C20561EE54954
:1096AA0075F00584FF24EFF582E43400F583E4F0D5
:1096BA0074042FF582E43401F583E4F0E490015A4E
:0896CA00F09001A1E014F02270
:10990A00E549B4651A755301755401755561E490BA
:10991A00018CF09001A17409F090015A7402F022AE
:109A8200E549B4690BC252E490015AF09001A1F089
:019A920022B1
:109AA300C252E490015AF0900159F09001A1F022C2
:10817F00789AE6600116900000E0600214F090001B
:10818F0001E0600214F0900002E0600214F0900031
:10819F000BE0600214F090000AE0600214F0789C8B
:1081AF0016E66003028252789C760A789BE660019D
:1081BF0016900004E0600214F0900005E0600214D5
:1081CF00F0900006E0600214F0900008E0600214E6
:1081DF00F0900009E0600214F078A0E660011690BC
:1081EF000003E0600214F09001E7E0600214F07801
:1081FF009D16E6704E789D760A90000CE060021492
:10820F00F078A2E61846600708E616187001169077
:10821F0001A3E0600214F09001A4E0600214F0905A
:10822F0001A7E0600214F0789E16E67016789E762D
:10823F000A789F16E6700C789F76069001A6E0608C
:04824F000214F02203
:106AF000535155452020434F53202053454E534575
:106B0000004F4E2020202020202020202020202048
:106B100020004F464620202020202020202020201A
:106B2000202000202020524550454154455220311C
:106B3000202020002020205245504541544552201D
:106B400032202020002020205245504541544552FB
:106B5000203320202000202020524550454154451C
:106B600052203420202000202020524550454154FE
:106B700045522035202020002020205245504541FC
:106B800054455220362020200020202052455045D8
:106B900041544552203720202000202020524550CB
:106BA00045415445522038202020002020205245C5
:106BB00050454154455220392020200020202052A9
:106BC000455045415445522031302020002020209E
:106BD000524550454154455220313120200020205B
:106BE000205245504541544552203132202000204A
:106BF0002020524550454154455220313320200039
:106C00002020205245504541544552203134202007
:106C10000020202052455045415445522031352016
:106C20002000202020524550454154455220313605
:106C3000202000202020524550454154455220310B
:106C400037202000202020524550454154455220F5
:106C500031382020002020205245504541544552D3
:106C600020313920200020202052455045415445F4
:076C70005220323020200009
:10002E00750C01E50CC394155018AF0C74182FF510
:10003E0082E43401F583E0FFEF60037F0122050CBB
:04004E0080E17F00CE
:01005200228B
:10904700205755128321EF6401704D90009AE0FF7D
:10905700EF24FF924D900158E0FF74422FF582E410
:109067003401F583E0FF90015BEFF0900158E0FFDA
:10907700742D2FF582E43401F583E0FF90015CEF56
:10908700F0900158E0FF90015DEFF012643090011D
:099097005EEFF0128538D23F2291
:108321009000E8E4F0A3E4F09000EBE4F0A3E4F0C3
:108331009000E7E4F09000E7E0FFEFC394154003FD
:108341000283C5900158E0FFEFD3941440069001D9
:10835100587401F0900158E0FF74182FF582E4344D
:1083610001F583E0FF9000EAEFF09000EAE0FFEF13
:10837100B40115900158E0FF74182FF582E434011F
:10838100F5837402F07F01229000EAE0FFEFB4026E
:10839100249000E8E0FEA3E0FFEF4E70189000E8A3
:1083A100E4F0A37401F0900158E0FF7E009000EB2F
:1083B100EEF0A3EFF0900158E004F09000E7E00444
:1083C100F00283369000E8E0FEA3E0FFEF4E700478
:1083D1007F0022229000ECE0FF900158EFF07F0136
:0183E1002279
:108253009000E8E4F0A3E4F09000EBE4F0A3E4F092
:108263009000E7E4F09000E7E0FFEFC394154003CC
:10827300028304900158E0FFEFD394144006900169
:10828300587401F0900158E0FF74182FF582E4341C
:1082930001F583E0FF9000EAEFF09000EAE0FFEFE2
:1082A300605090005BE0FF900158E0FEEE6F60428B
:1082B3009000EAE0FFEFB40115900158E0FF741855
:1082C3002FF582E43401F5837402F07F01229000DC
:1082D300E8E0FEA3E0FFEF4E7018900158E0FF7E48
:1082E300009000EBEEF0A3EFF09000E8E4F0A3744D
:1082F30001F0900158E004F09000E7E004F00282FE
:10830300689000E8E0FEA3E0FFEF4E70047F0022D8
:0E831300229000ECE0FF900158EFF07F012275
:1064300090005BE0FFEFD3941440037F2022900193
:10644000EDE4F09001ECE4F090005BE0FF9001EAF5
:10645000EFF0900095E0FFEFD3940650030265241F
:106460009001EBE4F09001EBE0FFEFC394154003E3
:1064700002651D9001EAE0FFEFB415069001EA7491
:1064800001F09001EAE0FF74EE2FF582E43400F5AC
:1064900083E0FFEF64FF70769001EAE0FF74BE2FA7
:1064A000F582E43400F583E0FF90005BE0FE74BE0B
:1064B0002EF582E43400F583E0FEEEC39F404F905A
:1064C000005BE0FF9001EAE0FEEEB507069001EA0E
:1064D000E0FF229001EAE0FF74BE2FF582E4340071
:1064E000F583E0FF9001ECE0FEEFD39E40209001A9
:1064F000EAE0FF9001EDEFF09001EAE0FF74BE2FBB
:10650000F582E43400F583E0FF9001ECEFF09001B8
:10651000EBE004F09001EAE004F00264659001ED24
:10652000E0FF22229001EBE4F09001EBE0FFEFC3EB
:10653000941540030265E09001EAE0FFEF700690D9
:1065400001EA7414F09001EAE0FF74EE2FF582E4A2
:106550003400F583E0FFEF64FF70769001EAE0FF1E
:1065600074BE2FF582E43400F583E0FF90005BE019
:10657000FE74BE2EF582E43400F583E0FEEEC39F88
:10658000404F90005BE0FF9001EAE0FEEEB50706A9
:106590009001EAE0FF229001EAE0FF74BE2FF5824D
:1065A000E43400F583E0FF9001ECE0FEEFD39E4081
:1065B000209001EAE0FF9001EDEFF09001EAE0FFAA
:1065C00074BE2FF582E43400F583E0FF9001ECEF18
:1065D000F09001EBE004F09001EAE014F00265298C
:0565E0009001EDE0FF59
:0165E5002293
:1069500090005BE0FFEFD3941440037F202290016E
:10696000F1E4F09001F0E4F0900095E0FFEFD394B3
:10697000065003026A3590005BE0FFEF04FF9001D0
:10698000EEEFF09001EFE4F09001EFE0FFEFC39441
:10699000154003026A2E9001EEE0FFEFD3941440FD
:1069A000069001EE7401F09001EEE0FF74EE2FF519
:1069B00082E43400F583E0FFEF64FF70629001EE43
:1069C000E0FF74BE2FF582E43400F583E0FF900011
:1069D0005BE0FE74BE2EF582E43400F583E0FEEE4B
:1069E000C39F403B9001EEE0FF74BE2FF582E4347C
:1069F00000F583E0FF9001F0E0FEEFD39E40209091
:106A000001EEE0FF9001F1EFF09001EEE0FF74BEC7
:106A10002FF582E43400F583E0FF9001F0EFF09071
:106A200001EFE004F09001EEE004F00269889001CB
:106A3000F1E0FF222290005BE0FFEF14FF9001EEF7
:106A4000EFF09001EFE4F09001EFE0FFEFC3941559
:106A50004003026AEA9001EEE0FFEF70069001EE5B
:106A60007414F09001EEE0FF74EE2FF582E4340030
:106A7000F583E0FFEF64FF70629001EEE0FF74BE0B
:106A80002FF582E43400F583E0FF90005BE0FE74B4
:106A9000BE2EF582E43400F583E0FEEEC39F403B5A
:106AA0009001EEE0FF74BE2FF582E43400F583E040
:106AB000FF9001F0E0FEEFD39E40209001EEE0FF5A
:106AC0009001F1EFF09001EEE0FF74BE2FF582E44B
:106AD0003400F583E0FF9001F0EFF09001EFE00467
:0F6AE000F09001EEE014F0026A479001F1E0FF40
:016AEF002284
:10679B0090005BE0FFEFD3941440037F2022900026
:1067AB0052E0FFEFB4FF0C900053E0FFEFB4FF0398
:1067BB007F00229001F5E4F09001F4E4F090009555
:1067CB00E0FFEFD39406500302689590005BE0FF67
:1067DB00EF04FF9001F2EFF09001F3E4F09001F37E
:1067EB00E0FFEFC39415400302688E9001F2E0FFC7
:1067FB00EFD3941440069001F27401F09001F2E093
:10680B00FF74EE2FF582E43400F583E0FFEF64FFB5
:10681B0070629001F2E0FF74BE2FF582E43400F554
:10682B0083E0FF90005BE0FE74BE2EF582E4340043
:10683B00F583E0FEEEC39F403B9001F2E0FF74BE98
:10684B002FF582E43400F583E0FF9001F4E0FEEFD6
:10685B00D39E40209001F2E0FF9001F5EFF0900104
:10686B00F2E0FF74BE2FF582E43400F583E0FF9075
:10687B0001F4EFF09001F3E004F09001F2E004F08A
:10688B000267E89001F5E0FF222290005BE0FFEF4A
:10689B0014FF9001F2EFF09001F3E4F09001F3E0BC
:1068AB00FFEFC39415400302694A9001F2E0FFEF3A
:1068BB0070069001F27414F09001F2E0FF74EE2F69
:1068CB00F582E43400F583E0FFEF64FF7062900122
:1068DB00F2E0FF74BE2FF582E43400F583E0FF9005
:1068EB00005BE0FE74BE2EF582E43400F583E0FE1F
:1068FB00EEC39F403B9001F2E0FF74BE2FF582E4A4
:10690B003400F583E0FF9001F4E0FEEFD39E4020CE
:10691B009001F2E0FF9001F5EFF09001F2E0FF74CF
:10692B00BE2FF582E43400F583E0FF9001F4EFF025
:10693B009001F3E004F09001F2E014F00268A790EC
:04694B0001F5E0FF73
:01694F002225
:109A370090005BE0FFEFD3941440037F2022900057
:049A47005BE0FF22BF
:10782000900157E0FFEFD394144006900157740184
:10783000F09000E7E4F0900157E0FF742D2FF582FF
:10784000E43401F583E0FF900157E0FE74032EF568
:1078500082E43401F583E0FEEEB50726900157E09F
:10786000FF74422FF582E43401F583E0FF90015765
:10787000E0FE74EE2EF582E43400F583E0FEEE6F58
:1078800060069000E77401F0900157E0FF74EE2F5E
:10789000F582E43400F583E0FF90005BE0FEEF6EDC
:1078A000600E90005BE0FF900157E0FEEE6F703AD3
:1078B0009000E7E0FFEF6043900157E0FFEFD394C3
:1078C000155014900157E0FF74182FF582E434012D
:1078D000F5837401F08024900157E0FF74182FF5B0
:1078E00082E43401F583E4F08011900157E0FF74E5
:1078F000182FF582E43401F583E4F09000E7E0FF0F
:10790000EF6044900157E0FF74032FF582E43401E7
:10791000F583E0FF900157E0FE742D2EF582E434EC
:1079200001F583EFF0900157E0FF74EE2FF582E44C
:107930003400F583E0FF900157E0FE74422EF5829B
:0E794000E43401F583EFF0900157E004F022EB
:1071F000900198E0FFEF600302729A900006E0FFB2
:10720000EF70037F0122129477EFB40103127960CB
:10721000204A037F0022129477EF64016003027317
:107220003A304A72C24A12709990004EE0FF9001C3
:1072300094EFF090004FE0FF900195EFF090004D3B
:10724000E0FF900196EFF0900196E0FFEFB41F147D
:10725000900192E0FF900195E0FEEEB507061279ED
:10726000667F0122900191E0FF900194E0FEEEB56F
:10727000070E900192E0FF900195E0FEEE6F60092D
:107280009001987401F07F002290008CE0FF900044
:1072900006EFF07F00227F002222900198E0FFEFAE
:1072A00064016003027333900006E0FFEF70037F18
:1072B0000122129477EFB40103127960204A037F10
:1072C0000022C24A12709990004EE0FF900194EFA4
:1072D000F090004FE0FF900195EFF090004DE0FF3F
:1072E000900196EFF0900196E0FFEFB41F1490012B
:1072F00092E0FF900195E0FEEEB507061279667FF9
:107300000122900191E0FF900194E0FEEEB507208C
:10731000900192E0FF900195E0FEEEB5071290001B
:107320008CE0FF900006EFF0900198E4F07F0022DF
:0B7330007F0022900198E4F07F002213
:10947700900083E0FFEF600D12798A40047F01803E
:10948700027F002222900084E0FFEF6013900085A6
:10949700E0FFE532D39F40047F0122227F00222292
:1094A700900085E0FFE532C39F50047F0122227FB1
:0294B700002291
:106F3D0090019DE0FFEF6003026FEF900008E0FF0E
:106F4D00EF70037F0122129477EFB401051279607F
:106F5D00800312796690019CE0FFEFB40106203B9F
:106F6D00037F002290019CE0FFEFB4020620410355
:106F7D007F0022129477EF6401706490019CE0FF12
:106F8D00EF64017021303B1EC23BE53F653E600959
:106F9D0090019D7401F07F0022900091E0FF900020
:106FAD0008EFF07F002290019CE0FFEF6402702F4C
:106FBD0030412CC24190019FE534F090019FE0FFDC
:106FCD0090019EE0FEEE6F600990019D7401F07FCF
:106FDD000022900091E0FF900008EFF07F00227FEB
:106FED00002290019DE0FFEF640160030270989014
:106FFD000008E0FFEF70037F0122129477EFB401D8
:10700D0005127960800312796690019CE0FFEFB460
:10701D000106203B037F002290019CE0FFEFB402AC
:10702D00062041037F0022129477EF6401705A907D
:10703D00019CE0FFEFB4011C303B19C23BE53FB5AD
:10704D003E1290019DE4F0900091E0FF900008EF5A
:10705D00F07F002290019CE0FFEF6402702B304125
:10706D0028C24190019FE534F090019FE0FF90010F
:10707D009EE0FEEEB5071290019DE4F0900091E0C8
:0C708D00FF900008EFF07F00227F00223F
:108DFF007BFF7A6A79F012973D12798A400B7BFFDD
:108E0F007A6B790112977280097BFF7A6B79121254
:108E1F0097727F17127D7BAF32127A31900054E038
:108E2F00FF127D4C900055E0FF127D4C900056E0F4
:108E3F00FF127D4C7F1C127D7BAF31127A31900077
:108E4F0054E0FF127D4C900055E0FF127D4C9000D6
:078E5F0056E0FF127D4C22DA
:10983C00900088E0FFEF6013900089E0FFE531D3E2
:10984C009F40047F0122227F002222900089E0FFAA
:0D985C00E531C39F50047F0122227F0022CE
:109AB300900083E0FFEF6004128AC022126C7722C9
:108AC0009001A5E0FFEF701612798A40729000863F
:108AD000E0FF90000AEFF09001A5E004F022900181
:108AE000A5E0FFEF6401702812798A401C90000A0B
:108AF000E0FFEF704AD25B900090E0FF900007EF3C
:108B0000F09001A5E004F022229001A5E4F02222D9
:108B10009001A5E0FFEFB4022112798A400B90008A
:108B200090E0FF900007EFF022900007E0FFEF7069
:108B30000EC25B9001A5E4F022229001A5E4F02290
:106C77009001A5E0FFEF704C900084E0FFEF6023E8
:106C8700900085E0FFE532D39F4013900086E0FF38
:106C970090000AEFF09001A5E004F0228026C25B85
:106CA700228021900085E0FFE532C39F50139000BA
:106CB70086E0FF90000AEFF09001A57403F02280B0
:106CC70003C25B229001A5E0FFEF640170359000DD
:106CD70085E0FFEF24FBFFE532D39F401F90000ABA
:106CE700E0FFEF6003026DDAD25B900087E0FF9070
:106CF700000BEFF09001A5E004F022229001A5E43B
:106D0700F022229001A5E0FFEF6402702E9000852B
:106D1700E0FFEF24FBFFE532D39F400B900087E0B5
:106D2700FF90000BEFF02290000BE0FFEF600302F3
:106D37006DDAC25B9001A5E4F022229001A5E0FF85
:106D4700EF64037043900085E0FF7E00EF2405FFAA
:106D5700EE3400FEAD327C00C3ED9FEE6480F8ECAC
:106D6700648098501C90000AE0FFEF7066D25B9039
:106D77000087E0FF90000BEFF09001A5E004F02200
:106D8700229001A5E4F022229001A5E0FFEF640420
:106D9700703C900085E0FF7E00EF2405FFEE340095
:106DA700FEAD327C00C3ED9FEE6480F8EC64809802
:106DB700500B900087E0FF90000BEFF02290000B44
:106DC700E0FFEF700EC25B9001A5E4F02222900174
:046DD700A5E4F0221D
:1099F40012679B8F1D9001E6E0FFEF651D600890E4
:079A040001E6E51DF0D25C54
:019A0B002238
:107B980090005BE0FFEF1285127BE1017BEB027B3B
:107BA800F5037BFF047C09057C13067C1D077C27F5
:107BB800087C31097C3B0A7C450B7C4F0C7C590DB9
:107BC8007C630E7C6D0F7C77107C81117C8B127C22
:107BD80095137C9F1400007CA87BFF7A6B79231295
:107BE8009772227BFF7A6B7934129772227BFF7A25
:107BF8006B7945129772227BFF7A6B7956129772CE
:107C0800227BFF7A6B7967129772227BFF7A6B79F6
:107C180078129772227BFF7A6B7989129772227B8E
:107C2800FF7A6B799A129772227BFF7A6B79AB1283
:107C38009772227BFF7A6B79BC129772227BFF7A4C
:107C48006B79CD129772227BFF7A6B79DE1297726D
:107C5800227BFF7A6B79EF129772227BFF7A6C791D
:107C680000129772227BFF7A6C7911129772227B2D
:107C7800FF7A6C7922129772227BFF7A6C79331221
:107C88009772227BFF7A6C7944129772227BFF7A73
:107C98006C7955129772227BFF7A6C79661297720B
:017CA80022B9
:10562E002020464C45582049562030303520202029
:10563E00002049502050524F4752414D4D494E4740
:10564E00200043544353532036332E302020202045
:10565E00202043544353532036372E302020202011
:10566E00202043544353532036392E3420202020FB
:10567E00202043544353532037312E3920202020ED
:10568E00202043544353532037342E3420202020DF
:10569E00202043544353532037372E3020202020D0
:1056AE00202043544353532037392E3720202020B7
:1056BE00202043544353532038322E3520202020AF
:1056CE00202043544353532038352E34202020209D
:1056DE00202043544353532038382E352020202089
:1056EE00202043544353532039312E35202020207F
:1056FE00202043544353532039342E382020202069
:10570E00202043544353532039372E342020202059
:10571E0020204354435353203130302E302020204C
:10572E0020204354435353203130332E3520202034
:10573E0020204354435353203130372E3220202023
:10574E0020204354435353203131302E3920202012
:10575E0020204354435353203131342E38202020FF
:10576E0020204354435353203131382E38202020EB
:10577E0020204354435353203132332E30202020E7
:10578E0020204354435353203132372E33202020D0
:10579E0020204354435353203133312E38202020C0
:1057AE0020204354435353203133362E35202020AE
:1057BE0020204354435353203134312E33202020A4
:1057CE0020204354435353203134362E3220202090
:1057DE0020204354435353203135312E3420202082
:1057EE0020204354435353203135362E372020206A
:1057FE0020204354435353203135392E3820202056
:10580E0020204354435353203136322E3220202051
:10581E0020204354435353203136352E352020203B
:10582E0020204354435353203136372E3920202025
:10583E0020204354435353203137312E3320202020
:10584E0020204354435353203137332E3820202009
:10585E0020204354435353203137372E33202020FA
:10586E0020204354435353203137392E39202020E2
:10587E0020204354435353203138332E35202020DB
:10588E0020204354435353203138362E32202020CB
:10589E0020204354435353203138392E39202020B1
:1058AE0020204354435353203139322E38202020A8
:1058BE0020204354435353203139362E3620202096
:1058CE0020204354435353203139392E3520202084
:1058DE0020204354435353203230332E3520202082
:1058EE0020204354435353203230362E352020206F
:1058FE0020204354435353203231302E3720202062
:10590E0020204354435353203231382E312020204F
:10591E0020204354435353203232352E372020203B
:10592E0020204354435353203232392E312020202D
:10593E0020204354435353203233332E362020201D
:10594E0020204354435353203234312E382020200C
:10595E0020204354435353203235302E3320202001
:10596E0020204354435353203235342E31202020EF
:10597E002020202020202020202020202020202019
:02598E002020D7
:1062740075840F1265E69001E87401F09001E974E9
:1062840003F07D007CFC7F10129537E49001E8F068
:106294009001E9F020A10875840F43E8C0800675D9
:1062A400840F53E83F129AC37BFF7A56792E1297D4
:1062B4003D129A0C900003741EF0900003E070FAF3
:1062C400129A7090005BE0FF6005D394144006902E
:1062D400005B7401F0127B981286FE128F8F128F6E
:1062E400EB1297A7D2AC127954900099E0FF78A1F1
:1062F400760008A6079000A4E09001A6F0E49000C0
:10630400EDF0900190F090018FF0900198F09001E1
:10631400A0F090005274FFF0900053F0E49001E676
:10632400F09001E5F0F558127966304313124ABF34
:10633400129A701286FE128F8F128FEBC24380EA7C
:1063440020A60E128DFFE4900190F090018FF08052
:10635400EF30461DC246124ABF129A701286FE12D0
:106364008F8F128FEB129AC3E490018FF0900190FB
:10637400F043E740305806128ECC1298C112422BDB
:106384001232DD1275B4E55BB45514E55CB4AA0FA2
:106394009001E77414F09001E7E070FA12795A90D2
:1063A40001A7E0703E12796C5039127A7A12782083
:1063B400125A74129AB3128F2F1299F4305C8130EE
:1063C4005D03026344C25C9001E6E02400FEE43411
:1063D400179001C2F0A3CEF09001BE7401F0D25D1B
:1063E400026344127954900099E0FF78A176000882
:1063F400A6079000A4E09001A6F0E49000EDF090D0
:106404000190F090018FF0900198F09001A0F0902D
:10641400005BE0900052F090005374FCF012796637
:0C6424007BFF7A56793F12973D026344DB
:108E660001AE01C901DA01EB01FC020E0220023358
:108E76000247025C02710287029902AB02C302DC5E
:108E860002F50310032B03480365038403A403C5FB
:108E960003E6040A042E04430453046A047A049184
:108EA60004A204BA04CC04E504F705100524053E23
:108EB6000552056D0582059E05D10605061C063B75
:068EC600067306AD06C7AD
:10998900C23DC23FEF25E02466F582E4348EF583BB
:0E999900E493F51A740193F51BD23ED23822E6
:09009600C23DC23FC23EC2382245
:0300A30002943490
:10943400C0E0C0F0C083C082C0D075D000C000C0FE
:1094440001C002C003C004C005C006C007205805FF
:109454001280AB80031290F6D007D006D005D0045A
:10946400D003D002D001D000D0D0D082D083D0F0AD
:03947400D0E03213
:03009300028CB923
:0B8CB900C0E0C0D075D000C006C007AE
:108CC400AE8430A704C2A78002D2A7758402E5331C
:108CD4007007AFBE75BB07802FE533B40107AFBE85
:108CE40075BB048023E533B40207AFBE75BB0680B1
:108CF40017E533B4030885BE3175BB04800AE53338
:108D0400B40409AFBE75BB0505338010E533B40563
:108D14000885BE3275BB048000753300C2ED8E84B5
:098D2400D007D006D0D0D0E03217
:030083000294FAEA
:1094FA00C0E0C0F0C083C082C0D075D000C000C038
:10950A0001C002C003C004C005C006C007C2CF1212
:10951A001D32D007D006D005D004D003D002D00126
:0D952A00D000D0D0D082D083D0F0D0E0327D
:03007300028822DE
:10882200C0E0C0F0C083C082C0D075D000C000C01C
:1088320001C002C003C004C005C006C007C2CF30D9
:108842005805128D9780031290A07897E660011662
:10885200304027C240D54A05754A0A054912747844
:10886200D51C09751C0A758401438820D5301875FA
:108872003060758402438820800DD240789816E6D5
:1088820070057604121A1A758401438810758402E1
:10889200D2ECD007D006D005D004D003D002D0014C
:0D88A200D000D0D0D082D083D0F0D0E03212
:03006B000292DD21
:1092DD00C0E0C0F0C083C082C0D075D000C000C057
:0D92ED0001C002C003C004C005C006C007D8
:0E92FA0085847412817F758402C28D85748410
:10930800D007D006D005D004D003D002D001D000B9
:0B931800D0D0D082D083D0F0D0E03263
:03005B000291F21D
:1091F200C0E0C0F0C083C082C0D075D000C000C043
:1092020001C002C003C004C005C006C0071259A9AC
:109212007899E6600116900007E0600214F0758408
:1092220001C28D127796D007D006D005D004D003A4
:10923200D002D001D000D0D0D082D083D0F0D0E004
:0192420032F9
:03005300029323F2
:10932300C0E0C0F0C083C082C0D075D000C000C010
:1093330001C002C003C004C005C006C007C28C3010
:109343005904C2598005D25912749AD007D006D055
:1093530005D004D003D002D001D000D0D0D082D029
:0693630083D0F0D0E032DF
:03002B00020016BA
:03001600C2CF3224
:03002300029A5EE0
:109A5E00309904C299C262309807859956C298D23D
:029A6E00613263
:03001B00020019C7
:0100190032B4
:10936900A984A2AF9264AEB1C2AF75840F53A1FEB6
:109379008FB1E4F5849001E8E042B79001E9E04259
:109389008F8C088D098D828C83EBF0E4F584900134
:10939900E9E0F4528F9001E8E0F452B78EB1898484
:0493A900A26492AF79
:0193AD00229D
:10953700A984A2AF9264AEB1C2AF8C088D098FB176
:10954700E4F5849001E8E0FF42B7E4F5849001E98F
:10955700E0FD428F850982850883E4F0EDF4528FA0
:0C956700EFF452B78EB18984A26492AF79
:0195730022D5
:10992A00AE84A2AF9264ABB1C2AF8FB18C0A8D0B79
:0F993A008D828C83E493FF8BB18E84A26492AFF5
:0199490022FB
:100EC800202020464C45582049562020202020200C
:100ED8000020202020202020202020202049444CB1
:100EE80045002054657374696E67204D6F646520F2
:100EF80020200043726F73732042757379204D6F01
:100F08006465200053656E642049646C654D6573A3
:100F1800736167650043726F73732042757379203C
:100F28004D6F6465310043726F7373204275737936
:100F3800204D6F6465320043726F7373204275737E
:100F480079204D6F6465330043726F737320427567
:100F58007379204D6F64653400202053656E646991
:100F68006E672043574944202000205741495420A8
:100F78005544544420464C414720004C5452564F47
:100F88004950204F5554474F494E470020564F4926
:100F980050204F5554474F494E47202000202049A4
:100FA8004E434F4D494E47204C545220200020209C
:100FB800494E434F4D494E472043544353532020F5
:100FC800002020494E434F4D494E4720444353206B
:100FD800200043544353532036332E302020202002
:100FE800202043544353532036372E3020202020CE
:100FF800202043544353532036392E3420202020B8
:10100800202043544353532037312E3920202020A9
:10101800202043544353532037342E34202020209B
:10102800202043544353532037372E30202020208C
:10103800202043544353532037392E372020202073
:10104800202043544353532038322E35202020206B
:10105800202043544353532038352E342020202059
:10106800202043544353532038382E352020202045
:10107800202043544353532039312E35202020203B
:10108800202043544353532039342E382020202025
:10109800202043544353532039372E342020202016
:1010A80020204354435353203130302E3020202009
:1010B80020204354435353203130332E35202020F1
:1010C80020204354435353203130372E32202020E0
:1010D80020204354435353203131302E39202020CF
:1010E80020204354435353203131342E38202020BC
:1010F80020204354435353203131382E38202020A8
:1011080020204354435353203132332E30202020A3
:1011180020204354435353203132372E332020208C
:1011280020204354435353203133312E382020207C
:1011380020204354435353203133362E352020206A
:1011480020204354435353203134312E3320202060
:1011580020204354435353203134362E322020204C
:1011680020204354435353203135312E342020203E
:1011780020204354435353203135362E3720202026
:1011880020204354435353203135392E3820202012
:1011980020204354435353203136322E322020200E
:1011A80020204354435353203136352E35202020F8
:1011B80020204354435353203136372E39202020E2
:1011C80020204354435353203137312E33202020DD
:1011D80020204354435353203137332E38202020C6
:1011E80020204354435353203137372E33202020B7
:1011F80020204354435353203137392E392020209F
:1012080020204354435353203138332E3520202097
:1012180020204354435353203138362E3220202087
:1012280020204354435353203138392E392020206D
:1012380020204354435353203139322E3820202064
:1012480020204354435353203139362E3620202052
:1012580020204354435353203139392E3520202040
:1012680020204354435353203230332E352020203E
:1012780020204354435353203230362E352020202B
:1012880020204354435353203231302E372020201E
:1012980020204354435353203231382E312020200C
:1012A80020204354435353203232352E37202020F8
:1012B80020204354435353203232392E31202020EA
:1012C80020204354435353203233332E36202020DA
:1012D80020204354435353203234312E38202020C9
:1012E80020204354435353203235302E33202020BE
:1012F80020204354435353203235342E31202020AC
:1013080020202020202020202020202020202020D5
:1013180020204443532030303620494E5620303266
:1013280031204443532030303720494E5620323143
:1013380034204443532030313520494E562031342F
:1013480031204443532030313720494E5620303520
:1013580030204443532030323120494E562030301B
:1013680036204443532030323320494E56203034FF
:1013780037204443532030323520494E56203234EA
:1013880034204443532030323620494E56203436D8
:1013980034204443532030333120494E56203632CE
:1013A80037204443532030333220494E56203035BD
:1013B80031204443532030333620494E56203137AC
:1013C80032204443532030343320494E562034349D
:1013D80035204443532030343720494E562030328C
:1013E80033204443532030353020494E5620303185
:1013F80037204443532030353120494E562030336E
:1014080032204443532030353320494E562034355A
:1014180032204443532030353420494E562034314D
:1014280033204443532030363520494E5620323736
:1014380031204443532030373120494E5620333031
:1014480036204443532030373220494E5620323418
:1014580035204443532030373320494E5620353009
:1014680036204443532030373420494E56203137F4
:1014780034204443532031313420494E56203731EB
:1014880032204443532031313520494E56203135DE
:1014980032204443532031313620494E56203735C7
:1014A80034204443532031323220494E56203232C0
:1014B80035204443532031323520494E56203336A7
:1014C80035204443532031333120494E562033369A
:1014D80034204443532031333220494E562035348A
:1014E80036204443532031333420494E562032327B
:1014F80033204443532031343120494E5620303173
:1015080035204443532031343320494E562034315A
:1015180032204443532031343520494E5620323747
:1015280034204443532031353220494E562031313E
:1015380035204443532031353520494E5620373322
:1015480031204443532031353620494E5620323617
:1015580035204443532031363220494E5620353009
:1015680033204443532031363520494E56203235F6
:1015780031204443532031373220494E56203033EE
:1015880036204443532031373420494E56203037D3
:1015980034204443532032303520494E56203236C9
:1015A80033204443532032313220494E56203335BC
:1015B80036204443532032313420494E56203030AF
:1015C80037204443532032323320494E562031339A
:1015D80034204443532032323520494E562031328C
:1015E80032204443532032323620494E562034317B
:1015F80031204443532032343320494E562033356A
:1016080031204443532032343420494E562030325E
:1016180035204443532032343520494E5620303744
:1016280032204443532032343620494E5620353236
:1016380033204443532032353120494E5620313629
:1016480035204443532032353220494E5620343613
:1016580032204443532032353520494E5620343405
:1016680036204443532032363120494E56203733F2
:1016780032204443532032363320494E56203230EC
:1016880035204443532032363520494E56203135D3
:1016980036204443532032363620494E56203435BE
:1016A80034204443532032373120494E56203036B7
:1016B80035204443532032373420494E56203134A4
:1016C80035204443532033303620494E5620303796
:1016D80031204443532033313120494E5620363689
:1016E80034204443532033313520494E5620343278
:1016F80033204443532033323520494E5620353267
:1017080036204443532033333120494E5620343653
:1017180035204443532033333220494E5620343544
:1017280035204443532033343320494E5620353333
:1017380032204443532033343620494E5620363124
:1017480032204443532033353120494E5620323419
:1017580033204443532033353620494E5620323106
:1017680032204443532033363420494E56203133F7
:1017780031204443532033363520494E56203132E8
:1017880035204443532033373120494E56203733D0
:1017980034204443532034313120494E56203232CC
:1017A80036204443532034313220494E56203134B8
:1017B80033204443532034313320494E56203035AA
:1017C80034204443532034323320494E5620333199
:1017D80035204443532034333120494E5620373284
:1017E80033204443532034333220494E5620353178
:1017F80036204443532034343520494E5620303463
:1018080033204443532034343620494E5620323551
:1018180035204443532034353220494E5620303544
:1018280033204443532034353420494E5620323631
:1018380036204443532034353520494E562033331F
:1018480032204443532034363220494E5620323514
:1018580032204443532034363420494E5620303207
:1018680036204443532034363520494E56203333EE
:1018780031204443532034363620494E56203636DC
:1018880032204443532035303320494E56203136D8
:1018980032204443532035303620494E56203037C5
:1018A80033204443532035313620494E56203433B3
:1018B80032204443532035323320494E56203234A7
:1018C80036204443532035323620494E5620333291
:1018D80035204443532035333220494E5620333483
:1018E80033204443532035343620494E5620313373
:1018F80032204443532035363520494E5620373060
:1019080033204443532036303620494E5620363350
:1019180031204443532036313220494E5620333447
:1019280036204443532036323420494E562036332D
:1019380032204443532036323720494E5620303324
:1019480031204443532036333120494E5620363017
:1019580036204443532036333220494E56203632FF
:1019680034204443532036353420494E56203734EA
:1019780033204443532036363220494E56203436DD
:1019880036204443532036363420494E56203331CE
:1019980031204443532037303320494E56203536C2
:1019A80035204443532037313220494E56203131B7
:1019B80034204443532037323320494E56203433A1
:1019C80031204443532037333120494E5620313596
:1019D80035204443532037333220494E562032367F
:1019E80031204443532037333420494E562033376F
:1019F80031204443532037343320494E562036355E
:101A080034204443532037353420494E5620313151
:021A1800362076
:107A7A009000B3E0FFB4010A90005274FFF0E402F0
:107A8A007B47EF64026003027B4C12794E787DE6F5
:107A9A006003027B3B305703027B3B900197E07007
:107AAA0032D23F90009AE024FF924D90005BE0FFB3
:107ABA0090015BF0900098E090015CF090015DEF1E
:107ACA00F012695090015EEFF012853890019774B8
:107ADA0002F022128253EF64017050D23F90015893
:107AEA00E0FF2442F582E43401F583E090015BF083
:107AFA00742D2FF582E43401F583E090015CF09057
:107B0A000158E090015DF012643090015EEFF09050
:107B1A00015BE024D2F582E43400F583E024FF928D
:107B2A004D128538900197E014F022900197E014E5
:107B3A00F090005BE0900052F0900098E0900053C3
:107B4A00F02290018FE0B40900503D907B5CF82848
:107B5A002873027B77027B7A027B7D027B80027B21
:107B6A0083027B86027B89027B8C027B8F0225340F
:107B7A000289360287910252C1024690022D700292
:0E7B8A003D46024ED0023845E490018FF022B5
:10253400900190E0B40C004003022D6A902547F806
:1025440028287302256B02259F02283B0228790262
:10255400289C0228C602298C022A16022AA9022AC9
:10256400D6022BA0022C75E49001E5F07BFF7A0ED5
:1025740079C812973D7BFF7A0E79D9129772900031
:102584005274FFF0900053F01279549000B4E0605C
:10259400031279789001907401F02220A55C1279DD
:1025A4004E9000B4E060031279729000B1E09000A4
:1025B40000F090005BE0FF900052F0900098E0FE85
:1025C400900053F09001907405F090015BEFF0904F
:1025D400015CEEF090005BE090015DF012643090DD
:1025E400015EEFF090009AE024FF924D128538D2FC
:1025F4003F7BFF7A0E79EA02973D9001E2E06403A3
:10260400703412794E9000B4E06003127972900035
:10261400B1E0900000F0E49001E2F09001E3E0907A
:102624000052F09001E4E0900053F0E4900190F047
:1026340090018F022A049001E2E0602D12794E90FD
:1026440000B4E060031279729000B1E0900000F0F1
:1026540090005BE0900052F090005374FEF0E49020
:102664000190F090018F022AA5129477EF64017013
:1026740061304A5EC24A90004EE0FFC39415505246
:1026840074D22FF582E43400F583E0FFA248E433EA
:102694006F703FA248924990004EE0900191F090F3
:1026A400004FE0900192F090004DE0900193F01201
:1026B4007099900193E0641F6018900191E0FF907D
:1026C4000192E0FD7C001285D390018F7402F00228
:1026D4002D6AC24A12002EBF011712794E9000B41F
:1026E400E060031279729000B1E0900000F0022AD9
:1026F400939000B5E06025129477EF6401600612B0
:10270400983CBF01177BFF7A0E79FB12973D90002E
:1027140092E078A0F69001907409F022129477EF79
:1027240064017068303B28C23B90019C04F0D239AC
:10273400853E3FE53F75F010A424DAF9740F35F0B7
:10274400FA7BFF12973DAF3F128BBFC239802A300C
:10275400413AC24190019EE534F075F010A4241A68
:10276400F9741335F0FA7BFF12973D90019EE0FF58
:102774001289BC90019C7402F090018F7405F0E4FE
:10278400900190F0900092E078A0F622C23BC24102
:1027940078A2E61846703F900099E060397BFF7A92
:1027A4000F790C12973D900099E0FF78A17600080C
:1027B400A60790005274FFF0900053F012794E90E7
:1027C40000B4E060031279729000B1E0900000F070
:1027D400900190022CF99000A4E0FF7003022D6F89
:1027E4009001A6E06003022D6F9000A2E0FE60104D
:1027F4007003022D6F9001A2E064016003022D6F4B
:102804009001A6EFF0E49001A2F012794E9000B48A
:10281400E060031279729000B1E0900000F0900043
:102824005BE0900052F090005374FDF0E49001904E
:10283400F090018F04F022900000E06003022D6FFD
:10284400305703022D6F90005BE0FF90015BF09026
:10285400015C74FFF090015DEFF090015EF0900078
:102864009AE024FF924D128538D23F12713B9001B9
:10287400907403F022787DE66003022D6F305703D5
:10288400022D6F127D95127DA490008DE0900001C1
:10289400F09001907404F022900001E06003022D96
:1028A4006F1279549000B4E06003127978E49001D7
:1028B40090F09001A204F090005274FFF090005345
:1028C400F02230A50302298990005BE0900052F0C9
:1028D400900098E0900053F0129477BF01051279AC
:1028E400608003127966787DE66003022D6F3057AD
:1028F40003022D6F900197E07034D23F90009AE06C
:1029040024FF924D90005BE0FF90015BF0900098F3
:10291400E090015CF090015DEFF012695090015E6F
:10292400EFF01285389001977402F002713B128225
:1029340053EF6401704CD23F900158E0FF2442F5FC
:1029440082E43401F583E090015BF0742D2FF5826D
:10295400E43401F583E090015CF0900158E09001CB
:102964005DF012643090015EEFF090015BE024D2E0
:10297400F582E43400F583E024FF924D1285380299
:102984002D4E022D4E022D6A900000E06003022DB0
:102994006F305703022D6F787DE66003022D6F9030
:1029A400005274FFF0900053F0128321EF64017021
:1029B40053900158E0FF2442F582E43401F583E0AA
:1029C40090015BF0742D2FF582E43401F583E090DF
:1029D400015CF0900158E090015DF0129A3790018B
:1029E4005EEFF090015BE024D2F582E43400F583DD
:1029F400E024FF924D128538D23F12713B90019032
:102A04007407F02290008DE0900001F09001900294
:102A14002AA5129477EF6401705F304A5EC24A902F
:102A2400004EE0FFC39415505274D22FF582E43463
:102A340000F583E0FFA248E4336F703F127099A25F
:102A440048924990004EE0900191F090004FE09040
:102A54000192F090004DE0900193F0641F601C908F
:102A64000191E0FF900192E0FD7C001285D3E49097
:102A74000190F090018F022CF9C24A787DE6600340
:102A8400022D6F305703022D6F12002EEF60079056
:102A940001907406F02290008DE0900001F0900106
:102AA400907408F022900001E06003022D6F127907
:102AB400549000B4E060031279789001A27401F09C
:102AC400E4900190F090005274FFF0900053F002F3
:102AD4007DA4129477EF64017063304A60C24A9017
:102AE400004EE0FFC39415505474D22FF582E434A1
:102AF40000F583E0FFA248E4336F7041A248924995
:102B040090004EE0900191F090004FE0900192F01F
:102B140090004DE0900193F0127099900193E0645D
:102B24001F601A900191E0FF900192E0FD7C001279
:102B340085D3E4900190F090018F022CF9C24A7879
:102B4400A0E66003022D6F90005BE0900052F090CD
:102B5400005374FDF09000B5E0FF64016004EFB42D
:102B64000215129477BF010F900093E0900005F0D6
:102B7400900190740AF0229000B5E0FF64036004B1
:102B8400EFB4041512983CBF010F900093E090003D
:102B940005F0900190740BF022022D6A129477BF15
:102BA4000108900093E0900005F0900005E07003A8
:102BB400022C899000B5E0B401097BFF7A0F791DDE
:102BC400022CA812794E7BFF7A0F792E1297727815
:102BD4007DE66003022D5B305703022D5B90019765
:102BE400E07031D23F90009AE024FF924D90005B58
:102BF400E0FF90015BF0900098E090015CF09001A0
:102C04005DEFF012695090015EEFF012853890018B
:102C140097022CF9128253EF6401704CD23F900159
:102C240058E0FF2442F582E43401F583E090015B2F
:102C3400F0742D2FF582E43401F583E090015CF00B
:102C4400900158E090015DF012643090015EEFF065
:102C540090015BE024D2F582E43400F583E024FFA4
:102C6400924D128538022D4E900197E014F0022DFA
:102C74005B12983CBF0108900093E0900005F0902F
:102C84000005E07012127954900099E0FF78A17663
:102C94000008A607022D6A9000B5E0B403097BFF83
:102CA4007A0F793F0297727BFF7A0F7950129772ED
:102CB40012794E787DE66003022D5B305703022DB6
:102CC4005B900197E07032D23F90009AE024FF922B
:102CD4004D90005BE0FF90015BF0900098E0900164
:102CE4005CF090015DEFF012695090015EEFF0121C
:102CF40085389001977402F022128253EF640170B8
:102D040050D23F900158E0FF2442F582E43401F5AB
:102D140083E090015BF0742D2FF582E43401F58398
:102D2400E090015CF0900158E090015DF012643095
:102D340090015EEFF090015BE024D2F582E4340070
:102D4400F583E024FF924D128538900197E014F04A
:102D540022900197E014F090005BE0900052F09014
:0C2D6400005374FDF022E4900190F02276
:10893600129047900190E0FF700C900000E0707577
:1089460090019004F022EF64017029205D1D9001D2
:10895600C27419F0A3E4F09001BE04F0D25D900158
:108966009004F07BFF7A0F796180067BFF7A0F799E
:1089760072029772900190E0FFB402189001E5E050
:1089860064017031F090008DE0900001F09001904C
:108996007403F022EFB40314900001E0701712790B
:1089A600549000B4E060051279788000E490018F5D
:0689B600F0900190F02298
:10879100900190E0703B900068E0602B12794E9060
:1087A10000B4E060031279729000B1E0900000F033
:1087B100900191E0900052F0900192E0900053F00E
:1087C1009001907401F022E4900190F090018FF0FB
:1087D10022900190E06401703E205D32900191E0B1
:1087E100FE900192E07C002400FFEC3E9001C2F07B
:1087F100A3EFF09001BE7401F0D25D900069E090AA
:10880100018F6004740480027403F0E4800E7BFF26
:108811007A0F7972029772E490018FF0900190F0D3
:018821002234
:1052C100900190E0704A900000E0600302562DA228
:1052D10049924D900191E090015BF0900192E09034
:1052E100015CF090005BE090015DF012695090016B
:1052F1005EEFF0128538D23F12713B90019774082E
:10530100F090008CE0900006F09001907401F02282
:10531100900190E06401703E1271F0EF60028055DF
:10532100787DE6600302562D30570302562D76280C
:10533100D257900197E014F0E0600302562D7402F9
:10534100F090008CE0900006F090008EE090000C50
:10535100F09001908069900190E064026003025432
:105361001E1271F0EF6002800C90008EE0600D90D3
:10537100000CE070079001907403F022787DE660E4
:105381000302562D30570302562D900197E07033DA
:10539100A249924D900191E090015BF0900192E061
:1053A10090015CF090005BE090015DF0126950901B
:1053B100015EEFF0128538D23F12713B9001977474
:1053C10002F022128253EF6401704F900158E0FF06
:1053D1002442F582E43401F583E090015BF0742D01
:1053E1002FF582E43401F583E090015CF0900158DF
:1053F100E090015DF012643090015EEFF090015B8E
:10540100E024D2F582E43400F583E024FF924D12CA
:105411008538D23F12713B0254D10254D190019090
:10542100E06403702E205D229001C2F0A374FFF0AE
:105431009001BE7401F0D25D127D95127966E490FF
:105441000198F09001907404F0227BFF7A0F797239
:10545100029772900190E064047043787DE66003E6
:1054610002562D30570302562DA249924D900191BB
:10547100E090015BF0900192E090015CF090015DA1
:10548100741FF0129A3790015EEFF0128538900187
:10549100977403F012713B9001907405F022900112
:1054A10090E0FF64057030787DE6600302562D3090
:1054B100570302562D900197E0700F90008DE090F8
:1054C1000001F09001907406F022787D7628D25781
:1054D100900197E014F022EF6406600302561690E3
:1054E10000B5E0601F303B0930410612983CEF7077
:1054F10013E490018FF0900190F0900092E078A079
:10550100F6025609305B7A304A77C24A90004EE083
:10551100FFC39415506B74D22FF582E43400F583E8
:10552100E0FFA248E4336F7058A248924990004EC0
:10553100E0900191F090004FE0900192F090004DC9
:10554100E0900193F0641F6038900191E0FFC394F3
:1055510015502E74D22FF582E43400F583E0FFA2BA
:1055610049E433B5071B900191E0FF900192E0FD02
:105571007C001285D390018F7402F0E4900190F0C9
:1055810022C24A787DE67055205752128321EF647A
:1055910001704A900158E0FF2442F582E43401F59C
:1055A10083E090015BF0742D2FF582E43401F583E3
:1055B100E090015CF0900158E090015DF0126430E0
:1055C10090015EEFF090015BE024D2F582E43400BB
:1055D100F583E024FF924D12853812713B90000152
:1055E100E070491279549000B4E060031279789028
:1055F100005274FFF0900053F09001A27401F0E4A6
:1056010090018FF0900190F0900099E0FF78A176E1
:105611000008A60722900190E0D39406400EE49082
:0D562100018FF0900190F078A1F608F622BC
:10469000900190E070107BFF7A0F798312973D9024
:1046A00001907401F022900190E064017059900033
:1046B00000E06003024ABEA249924D900191E09051
:1046C000015BF0900192E090015CF090005BE09063
:1046D000015DF012695090015EEFF0128538D23F13
:1046E00012713B90008CE0900006F090008EE090FC
:1046F000000CF09000B8E09001A3F09001977403D3
:10470000F090019014F022900190E0FF6402702973
:10471000787DE66003024ABE305703024ABE76281F
:10472000D257900197E014F0E06003024ABE740291
:10473000F090019004F0C24A22EF64036003024843
:1047400036129AB3205B089000B8E07002803F9068
:1047500000B8E0FF60089001A3E070028030305B99
:104760000D304A0A9001A3EFF0C24A127960129408
:1047700077EF70031279669001E5E0B40104E4027A
:10478000485B90008EE0600D90000CE07007900197
:10479000907404F022787DE66003024ABE3057032D
:1047A000024ABE900197E07033A249924D90019168
:1047B000E090015BF0900192E090015CF090005B72
:1047C000E090015DF012695090015EEFF0128538C3
:1047D000D23F12713B9001977402F022128253EF84
:1047E0006401704F900158E0FF2442F582E43401E7
:1047F000F583E090015BF0742D2FF582E43401F530
:1048000083E090015CF0900158E090015DF012644B
:104810003090015EEFF090015BE024D2F582E43449
:1048200000F583E024FF924D128538D23F12713B90
:104830000248E90248E9900190E06404702E205D8E
:10484000229001C2F0A374FFF09001BE7401F0D277
:104850005D127D95127966E4900198F09001907454
:1048600005F0227BFF7A0F7972029772900190E037
:1048700064057043787DE66003024ABE3057030248
:104880004ABEA249924D900191E090015BF09001E7
:1048900092E090015CF090015D741FF0129A3790E5
:1048A000015EEFF01285389001977403F012713BAE
:1048B0009001907406F022900190E0FF6406703041
:1048C000787DE66003024ABE305703024ABE90017B
:1048D00097E0700F90008DE0900001F090019074CF
:1048E00007F022787D7628D257900197E014F022C5
:1048F000EF64076003024AA79000B5E0601F303BF9
:104900000930410612983CEF7013E490018FF0904B
:104910000190F0900092E078A0F6024A9A12947703
:10492000EF64016003024A0490008DE0900001F002
:10493000204A03024A04C24A129477EF64016003DA
:10494000024A04900191E0FF90004EE0FEB507128C
:1049500090004FE0FF900192E0B50706E4900195CA
:10496000F022EEC394154003024A0490004EE0FF8B
:1049700024D2F582E43400F583E0FEA248E4336EED
:104980006003024A04900195E0FE701BA248924920
:10499000900194EFF090004FE0900195F090004D61
:1049A000E0900196F0805D90004EE0FF6E7055A2A1
:1049B000489249900191EFF090004FE0900192F001
:1049C00090004DE0900193F0641F6038900191E0F9
:1049D000FFC39415502E74D22FF582E43400F58372
:1049E000E0FFA249E433B5071B900191E0FF90017D
:1049F00092E0FD7C001285D390018F7402F0E49068
:104A00000190F022787DE6706020575D128321EFDF
:104A100064017055900158E0FF2442F582E43401AE
:104A2000F583E090015BF0742D2FF582E43401F5FD
:104A300083E090015CF0900158E090015DF0126419
:104A40003090015EEFF090015BE024D2F582E43417
:104A500000F583E024FF924D128538900190740692
:104A6000F0E490018FF012713B900001E070381279
:104A700079549000B4E0600312797890005274FF8A
:104A8000F0900053F09001A27401F0E490018FF0D7
:104A9000900190F0127D95127DA4900099E0FF782E
:104AA000A1760008A60722900190E0D39407400E5B
:0F4AB000E490018FF0900190F078A1F608F622C3
:102D7000900190E06003022E4F129477EF6401708F
:102D800057304A54C24A90004EE0FFC39415504851
:102D900074D22FF582E43400F583E0FFA248E433D7
:102DA0006F7035127099A248924990004EE09001E0
:102DB00091F090004FE0900192F090004DE0900172
:102DC00093F0641F6012900191E0FF900192E0FD8A
:102DD0007C001285D30231ABC24A78A0E6600302C0
:102DE00032DC129477EF6401705390005EE070243F
:102DF0001279549000B4E060031279789000B5E045
:102E0000B4010F90005BE0900052F090005374FE0C
:102E1000F022803512794E9000B4E060031279728E
:102E20009000B1E0900000F090005BE0900052F064
:102E300090005374FEF09001907401F022127954C6
:102E40009000B4E06003127978C239E40232D8907D
:102E50000190E064017061305D03022FB090019C2D
:102E6000E0FBB4010FE53F2400FEE434159001C2FD
:102E7000F0A3CEF0EBB4021190019EE02400FEE43A
:102E800034169001C2F0A3CEF09001BE7401F0D2CE
:102E90005D90008EE090000CF0900091E0900008B2
:102EA000F0900060E0600BE4900190F090018F02E0
:102EB0002FD89001900232CC900190E06402707A99
:102EC000900000E060030232DC90019CE06401703D
:102ED00025AF3F129989E53F75F010A424DAF97403
:102EE0000F35F0FA7BFF12973DE53F75F010A424F3
:102EF000DAF9740F803590019CE0640260030232BD
:102F0000DC90019EE0FF121EB790019EE075F0106C
:102F1000A4241AF9741335F0FA7BFF12973D90013F
:102F20009EE075F010A4241AF9741335F0FA7BFFB3
:102F30001297729001907403F022900190E0640364
:102F40007024126F3DEF6002801290008EE07003DB
:102F50000232DC90000CE060030232DC127D9590BE
:102F600001907404F022900190E06404704B205DA5
:102F70003F9001C2F0A374FFF09001BE7401F0D243
:102F80005D127DA4127966E490019DF090005DE0F1
:102F9000600E90009FE0900009F090019002325B7B
:102FA0009000A0E0900002F012009690019080281E
:102FB0007BFF7A0F7972029772900190E06405604E
:102FC000030230BF900009E070121200969000A03A
:102FD000E0900002F09001907406F022129477EFD6
:102FE0006401706B120096303B30C23B90019C74C0
:102FF00001F0853E3FC239E53F75F010A424DAF9AF
:10300000740F35F0FA7BFF12973DAF3F128BBFE490
:10301000900190F090018F02325B304132C24190BA
:10302000019EE534F075F010A4241AF9741335F0FC
:10303000FA7BFF12973D90019EE0FF1289BC900140
:103040009C7402F0E4900190F090018F02325BC218
:103050003BC241129477EF64017061304A5E120006
:1030600096C239C24A90004EE0FFC39415504D7489
:10307000D22FF582E43400F583E0FFA248E4336FF9
:10308000703A127099A248924990004EE0900191D6
:10309000F090004FE0900192F090004DE09001938D
:1030A000F0641F6017900191E0FF900192E0FD7CB9
:1030B000001285D390018F740202313CC24A2290E3
:1030C0000190E0640660030231B4900002E07007F2
:1030D0009001907407F022129477EF6401706230CF
:1030E0003B2BC23B90019C04F0853E3FC239E53F3B
:1030F00075F010A424DAF9740F35F0FA7BFF1297FB
:103100003DAF3F128BBF90018F7405802F3041314E
:10311000C24190019EE534F075F010A4241AF974B0
:103120001335F0FA7BFF12973D90019EE0FF128964
:10313000BC90019C7402F090018F7405F0E40231A0
:10314000EDC23BC241129477EF64017064304A6172
:10315000120096C239C24A90004EE0FFC394155047
:103160005074D22FF582E43400F583E0FFA248E4E6
:10317000336F703D127099A248924990004EE090D2
:103180000191F090004FE0900192F090004DE0909E
:103190000193F0641F601A900191E0FF900192E0AA
:1031A000FD7C001285D3E4900190F090018F0232F3
:1031B000CCC24A22900190E0640760030232D390AF
:1031C0000001E0702D1279549000B4E06003127990
:1031D00078127DA4900099E0FF78A1760008A607F8
:1031E0009001A27401F0C239E490018FF090019037
:1031F000F022129477EF64017065303B2CC23B9053
:10320000019C04F0853E3FE53F75F010A424DAF9F7
:10321000740F35F0FA7BFF12973DAF3F128BBFE47E
:10322000900190F090018F8032304133C241900183
:103230009EE534F075F010A4241AF9741335F0FAF1
:103240007BFF12973D90019EE0FF1289BC90019C8C
:103250007402F0E4900190F090018F7405F022C2A6
:103260003BC241129477EF64017065304A621200EC
:1032700096C239C24A90004EE0FFC3941550517473
:10328000D22FF582E43400F583E0FFA248E4336FE7
:10329000703E127099A248924990004EE0900191C0
:1032A000F090004FE0900192F090004DE09001937B
:1032B000F0641F601B900191E0FF900192E0FD7CA3
:1032C000001285D3E4900190F090018F7402F022F7
:0D32D000C24A22E4900190F090018FF0229C
:103D4600900190E070107BFF7A0F799412973D9066
:103D560001907401F022900190E06401706090007F
:103D660000E0600302422A90008EE090000CF09082
:103D760000B8E09001A3F090019CE0B40112AF3FBF
:103D8600129989E53F75F010A424DAF9740F8020A2
:103D960090019CE06402600302422A90019EE0FFCB
:103DA600121EB790019EE075F010A4241AF9741340
:103DB60035F0FA7BFF12977290019002421A900139
:103DC60090E064026003023E54129AB3205B0890AE
:103DD60000B8E07002800C9000B8E0600B9001A380
:103DE600E07005127966805F305B329000B8E09033
:103DF60001A3F090019CE0B4010D303B0AE53FB50C
:103E06003E05C23B12796090019CE0B4020F30413E
:103E16000C90019EE0B53405C24112796012947788
:103E2600EF70031279669001E5E0B40105127D9505
:103E3600803790008EE0700302422A90000CE0600A
:103E46000302422A127D959001907403F02290019C
:103E560090E0B40324205D189001C2E4F0A374FF3F
:103E6600F09001BE7401F0D25D9001907404F022CE
:103E76007BFF7A0F7972029772900190E06404706A
:103E86002C127DA4127966E490019DF090005DE00D
:103E9600600E90009FE0900009F09001900241763C
:103EA6009000A0E0900002F0120096801C90019015
:103EB600E064056003023FD0900009E07012120032
:103EC600969000A0E0900002F09001907406F02217
:103ED600129477EF64016003023F60120096303B54
:103EE60039C23BE53F653E700302422A90019C744D
:103EF60001F0853E3FC239E53F75F010A424DAF99A
:103F0600740F35F0FA7BFF12973DAF3F128BBFE47B
:103F1600900190F090018F02417630413DC2419070
:103F2600019EE06534700302422A90019EE534F05A
:103F360075F010A4241AF9741335F0FA7BFF129762
:103F46003D90019EE0FF1289BC90019C7402F0E452
:103F5600900190F090018F024176C23BC2411294CB
:103F660077EF64017061304A5E120096C239C24A28
:103F760090004EE0FFC39415504D74D22FF582E4A5
:103F86003400F583E0FFA248E4336F703A1270996B
:103F9600A248924990004EE0900191F090004FE0C7
:103FA600900192F090004DE0900193F0641F60172D
:103FB600900191E0FF900192E0FD7C001285D39084
:103FC600018F740202406AC24A22900190E06406A0
:103FD60060030240E2900002E0700F90008DE090D6
:103FE6000001F09001907407F022129477EF6401BB
:103FF6007077303B35C23BE53F653E700302422A8F
:1040060090019C7401F0853E3FC239E53F75F01082
:10401600A424DAF9740F35F0FA7BFF12973DAF3F0F
:10402600128BBF90018F7405803A30413CC241909B
:10403600019EE06534700302422A90019EE534F049
:1040460075F010A4241AF9741335F0FA7BFF129751
:104056003D90019EE0FF1289BC90019C7402F09095
:10406600018F7405F0E40241ACC23BC24112947761
:10407600EF64017064304A61120096C239C24A90F8
:10408600004EE0FFC39415505074D22FF582E434ED
:1040960000F583E0FFA248E4336F703D127099A2E9
:1040A60048924990004EE0900191F090004FE090C8
:1040B6000192F090004DE0900193F0641F601A9019
:1040C6000191E0FF900192E0FD7C001285D3E4901F
:1040D6000190F090018F02421AC24A22900190E0AC
:1040E60064076003024221129477EF6401600302C1
:1040F600417A90008DE0900001F0303B36C23BE5FE
:104106003F653E700302422A90019C7401F0853E91
:104116003FE53F75F010A424DAF9740F35F0FA7B09
:10412600FF12973DAF3F128BBFE4900190F09001D4
:104136008F803D30413EC24190019EE06534700360
:1041460002422A90019EE534F075F010A4241AF973
:10415600741335F0FA7BFF12973D90019EE0FF1233
:1041660089BC90019C7402F0E4900190F090018F5C
:104176007405F022C23BC241900001E0702D127915
:10418600549000B4E06003127978127DA4900099EF
:10419600E0FF78A1760008A6079001A27401F0C29C
:1041A60039E490018FF0900190F022129477EF6439
:1041B600017065304A62120096C239C24A90004EBA
:1041C600E0FFC39415505174D22FF582E43400F504
:1041D60083E0FFA248E4336F703E127099A24892C2
:1041E6004990004EE0900191F090004FE0900192CE
:1041F600F090004DE0900193F0641F601B900191D8
:10420600E0FF900192E0FD7C001285D3E4900190DE
:10421600F090018F7402F022C24A22E4900190F0DD
:0542260090018FF02261
:104ED000900190E070469001E3E0900052F0900164
:104EE000E4E0900053F07BFF7A0F79A512973DE440
:104EF0009001E2F0900052E0FF900053E0FD7C0052
:104F00001285D3900052E024D2F582E43400F58378
:104F1000E024FF92499001907401F022900190E00A
:104F20006401704B900000E060030252C0A24992FD
:104F30004D9001E3E090015BF09001E4E090015CB2
:104F4000F090005BE090015DF012695090015EEF1F
:104F5000F0128538D23F12713B900082E09001A49C
:104F6000F090008EE090000CF09001900252B09012
:104F70000190E064026003025070129AB3305B103B
:104F8000304A0D900082E09001A4F0C24A1279608C
:104F9000129477EF70031279669001E5E0B4010C8A
:104FA000E4F0127D959001907404F0229001A4E049
:104FB0007008900082E06002800C90008EE060102B
:104FC00090000CE0700A127D959001907403F0221D
:104FD000787DE660030252C03057030252C0900150
:104FE00097E07032A249924D9001E3E090015BF0AE
:104FF0009001E4E090015CF090005BE090015DF0D6
:1050000012695090015EEFF0128538D23F12713B69
:105010009001970252B0128253EF6401704F9001D9
:1050200058E0FF2442F582E43401F583E090015B0F
:10503000F0742D2FF582E43401F583E090015CF0EB
:10504000900158E090015DF012643090015EEFF045
:1050500090015BE024D2F582E43400F583E024FF84
:10506000924D128538D23F12713B02511D02511DE3
:10507000900190E0B40323205D179001C2E4F0A3F7
:1050800074FFF09001BE7401F0D25D900190740441
:10509000F07BFF7A0F7972029772900190E06404BE
:1050A0007049127DA4127966787DE660030252C0D1
:1050B0003057030252C0A249924D900191E09001F5
:1050C0005BF0900192E090015CF090015D741FF044
:1050D000129A3790015EEFF01285389001977403B1
:1050E000F012713B9001907405F022900190E0FF66
:1050F00064057030787DE660030252C030570302C9
:1051000052C0900197E0700F90008DE0900001F088
:105110009001907406F022787D7628D257900197FE
:10512000E014F022EF640660030252B7900001E041
:10513000702A1279549000B4E06003127978127DDD
:10514000A4900099E0FF78A1760008A6079001A23C
:105150007401F0C239E490018FF08069129477EF06
:1051600064017066303B2DC23B90019C04F0853E8B
:105170003FC239E53F75F010A424DAF9740F35F019
:10518000FA7BFF12973DAF3F128BBF90018F7405E2
:10519000F0E48031304133C24190019EE534F07536
:1051A000F010A4241AF9741335F0FA7BFF12973D1E
:1051B00090019EE0FF1289BC90019C7402F0900166
:1051C0008F7405F0E4900190F022C23BC24112942A
:1051D00077EF640160030252B490008DE09000010B
:1051E000F0204A030252B4120096C239C24A90011A
:1051F00091E0FF90004EE0FEB5071290004FE0FFF7
:10520000900192E0B50706E4900195F022EEC39478
:105210001540030252B490004EE0FF24D2F582E420
:105220003400F583E0FEA248E4336E60030252B41A
:10523000900195E0FE701BA2489249900194EFF016
:1052400090004FE0900195F090004DE0900196F0B5
:10525000806290004EE06E705B127099A248924995
:1052600090004EE0900191F090004FE0900192F09C
:1052700090004DE0900193F0641F6038900191E040
:10528000FFC39415502E74D22FF582E43400F583B9
:10529000E0FFA249E433B5071B900191E0FF9001C4
:1052A00092E0FD7C001285D3E4900190F090018F94
:1052B0007402F022C24A22E4900190F090018FF033
:0152C00022CB
:10384500900190E0706390005BE0900052F0900072
:103855005374FEF09001E2E0B4011D9001E4E0F53F
:103865003F7BFF7A0F79B612973D9001E4E0FF1296
:103875008BBF90019C7401F09001E2E0B4021F90AF
:1038850001E4E090019EF07BFF7A0F79C912973D24
:103895009001E4E0FF1289BC90019C7402F0E49071
:1038A50001E2F090019004F022900190E064017033
:1038B50058900000E06003023D4590008EE09000C6
:1038C5000CF090019CE0B40112AF3F129989E53FDD
:1038D50075F010A424DAF9740F802090019CE0643F
:1038E500026003023D4590019EE0FF121EB7900164
:1038F5009EE075F010A4241AF9741335F0FA7BFFD5
:10390500129772900190023D35900190E06402702B
:1039150061129AB3305B2A90019CE0B4010D303BF3
:103925000AE53FB53E05C23B12796090019CE0B4C3
:10393500020F30410C90019EE0B53405C241127969
:1039450060129477EF70031279669001E5E0B40197
:1039550005127D95803790008EE07003023D4590FD
:10396500000CE06003023D45127D959001907403C3
:10397500F022900190E0B40324205D189001C2E488
:10398500F0A374FFF09001BE7401F0D25D90019038
:103995007404F0227BFF7A0F79720297729001907E
:1039A500E064047027127DA412796690005DE060E2
:1039B5000E90009FE0900009F0900190023CC490A9
:1039C50000A0E0900002F0120096801C900190E0AB
:1039D50064056003023AEE900009E0701212009649
:1039E5009000A0E0900002F09001907406F0221281
:1039F5009477EF64016003023A7E120096303B39FA
:103A0500C23BE53F653E7003023D4590019C740154
:103A1500F0853E3FC239E53F75F010A424DAF9740C
:103A25000F35F0FA7BFF12973DAF3F128BBFE49045
:103A35000190F090018F023CC430413DC24190019C
:103A45009EE065347003023D4590019EE534F075B6
:103A5500F010A4241AF9741335F0FA7BFF12973D80
:103A650090019EE0FF1289BC90019C7402F0E490E5
:103A75000190F090018F023CC4C23BC24112947781
:103A8500EF64017061304A5E120096C239C24A90F5
:103A9500004EE0FFC39415504D74D22FF582E434E7
:103AA50000F583E0FFA248E4336F703A127099A2E3
:103AB50048924990004EE0900191F090004FE090BF
:103AC5000192F090004DE0900193F0641F60179013
:103AD5000191E0FF900192E0FD7C001285D39001F9
:103AE5008F7402023B88C24A22900190E06406600E
:103AF50003023C00900002E0700F90008DE0900002
:103B050001F09001907407F022129477EF64017030
:103B150077303B35C23BE53F653E7003023D45903E
:103B2500019C7401F0853E3FC239E53F75F010A454
:103B350024DAF9740F35F0FA7BFF12973DAF3F1287
:103B45008BBF90018F7405803A30413CC241900192
:103B55009EE065347003023D4590019EE534F075A5
:103B6500F010A4241AF9741335F0FA7BFF12973D6F
:103B750090019EE0FF1289BC90019C7402F09001B7
:103B85008F7405F0E4023C36C23BC241129477EFD4
:103B950064017064304A61120096C239C24A9000CD
:103BA5004EE0FFC39415505074D22FF582E43400D3
:103BB500F583E0FFA248E4336F703D127099A24887
:103BC500924990004EE0900191F090004FE09001F5
:103BD50092F090004DE0900193F0641F601A9001FF
:103BE50091E0FF900192E0FD7C001285D3E4900105
:103BF50090F090018F023D35C24A22900190E06419
:103C0500076003023D3C900001E0702A1279549050
:103C150000B4E06003127978900099E0FF78A1760E
:103C25000008A6079001A27401F0C239E490018F43
:103C3500F0900190F022129477EF64016003023C4A
:103C4500C890008DE0900001F0303B36C23BE53F67
:103C5500653E7003023D4590019C7401F0853E3F31
:103C6500E53F75F010A424DAF9740F35F0FA7BFFFF
:103C750012973DAF3F128BBFE4900190F090018FFA
:103C8500803D30413EC24190019EE06534700302A3
:103C95003D4590019EE534F075F010A4241AF974A1
:103CA5001335F0FA7BFF12973D90019EE0FF1289D4
:103CB500BC90019C7402F0E4900190F090018F7427
:103CC50005F022C23BC241129477EF640170653062
:103CD5004A62120096C239C24A90004EE0FFC39470
:103CE50015505174D22FF582E43400F583E0FFA21C
:103CF50048E4336F703E127099A248924990004E85
:103D0500E0900191F090004FE0900192F090004D0D
:103D1500E0900193F0641F601B900191E0FF90011A
:103D250092E0FD7C001285D3E4900190F090018F24
:103D35007402F022C24A22E4900190F090018FF0C3
:013D4500225B
:1000A600202020202020202020202020202020204A
:1000B6005245504541544552204E554D42455220D9
:1000C6002020202020202020203120746F20323054
:1000D600202053495445204E554D4245522020205C
:1000E6002020202020202020203120746F20393924
:1000F6008202001101021501148202011103041586
:1001060001632020202020202020202020202020C5
:1001160020202020202020202020202020202020D9
:10012600202020434F5552544553592042454550AF
:100136002020204354435353204F4E2048414E47DE
:10014600202020205553455220454E41424C452003
:10015600202020205245534552564520544F4E45A7
:10016600202020204E4554574F524B204D4F44459A
:100176002020204E4554574F524B204E554D424558
:100186005220202020202020202020202020202037
:100196002020202020202020202020202020202059
:1001A6002020202020202020202020202020202049
:1001B6002020202020202020202020202020202039
:1001C6002020202020202020202020202020313DFB
:1001D600454E2020202020202020202020204D4F6A
:1001E6004445202020202020202020202020544F5D
:1001F6004E4564010011020C150001640200110352
:100206000C15000164040011040C150001640800BB
:1002160011050C15000164100011060D150002C829
:10022600030111070A190101202020202020202087
:1002360020202020202020202020202020202020B8
:10024600202020202020202020434F555254455363
:100256005920424545502020204354435353204FB4
:100266004E2048414E4720202020555345522045D8
:100276004E41424C4520202020205245534552569F
:100286004520544F4E45202020204E4554574F526E
:100296004B204D4F44452020204E4554574F524B3E
:1002A600204E554D4245522020202020202020203F
:1002B6002020202020202020202020202020202038
:1002C6002020202020202020202020202020202028
:1002D6002020202020202020202020202020202018
:1002E6002020202020202020202020202020202008
:1002F60020202020313D454E202020202020202077
:10030600202020204D4F4445202020202020202042
:1003160020202020544F4E4564010011020C150088
:100326000164020011030C15000164040011040CA1
:1003360015000164080011050C1500016410001178
:10034600060D150001C8030111070A190101202035
:100356002020202020202020202020202020202097
:100366002020202020202020202020202020204364
:100376004F55525445535920424545502020202080
:100386005553455220454E41424C4520202020439E
:10039600524F535320544F4E45204D4F4445204312
:1003A600544353532F4443532043524F5353202017
:1003B6004E4554574F524B204D4F44452020204E1A
:1003C6004554574F524B204E554D42455220202002
:1003D6002020202020202020202020202020202017
:1003E60020202020202020202020313D454E202086
:1003F600202020202020202020204D4F4445202052
:1004060020202020202020202020544F4E45202030
:1004160020202020202020202020202020206401B1
:1004260000110209150001640200110309150001FB
:1004360064040011060A150001C8030111070C190E
:1004460001012020202020202020202020202020E4
:100456002020202020202020202020202020202096
:10046600202001010101010101010100000000003D
:100476000000000000000000000000000000000076
:100486000000000000000000000000000000000066
:100496000000000000000000000000000000000056
:1004A6000000000000000000000000000000000046
:1004B60000000000000000000000000020202020B6
:1004C6002020202020202020202020202020202026
:1004D6002020202020202020202020200101010192
:1004E6000101010101000000000000000000000001
:1004F60000000000000000000000000000000000F6
:1005060000000000000000000000000000000000E5
:1005160000000000000000000000000000000000D5
:1005260000000000000000000000000000000000C5
:100536000000000000002020202020202020202075
:1005460020202020202020202020202020202020A5
:1005560020202020202001010101010101010120AC
:100566002020202020202020202020202020202085
:100576002020202020202020202020202020202075
:1005860054454C434F2050524F4752414D20202056
:10059600524144494F2050524F4752414D2020204E
:1005A60050484F4E452050524F4752414D20202033
:1005B600434F4D50552050524F4752414D20202019
:1005C6002041434345535320434F44452020204474
:1005D600544D462054454C434F204C4556454C44BB
:1005E600544D4620524144494F204C4556454C42B5
:1005F60045455020524144494F204C4556454C42B2
:100606004545502054454C434F204C4556454C4398
:1006160057494420524144494F204C4556454C5673
:100626004F49434520524144494F204C45564C566C
:100636004F4943452054454C434F204C45564C505A
:1006460041474520524144494F204C4556454C436D
:100656005443535320524144494F204C45564C4431
:10066600435320524144494F204C4556454C204C5B
:10067600545220524144494F204C4556454C205235
:10068600505420524144494F204C4556454C205425
:10069600454C434F20524144494F204C45564C52FD
:1006A6004144494F2054454C434F204C45564C52EB
:1006B6004144494F204C494D4954204C45564C2005
:1006C600434F53204F5220535155454C4348202009
:1006D60020434F5320504F4C4152495459202043F8
:1006E6004F53205452494747455220564F4C544386
:1006F6004F5320414351554953542054494D454386
:100706004F532052454C454153452054494D4520B1
:1007160053454E534520504F4C415249545920534E
:10072600454E205452494747455220564F4C545344
:10073600454E20414351554953542054494D455344
:10074600454E2052454C454153452054494D452080
:100756004C545220484F4C442044454C415920505B
:100766005454205455524E4F46462054494D4552F6
:10077600455045415445522054494D454F55542006
:1007860020414E54492D4B45524348554E4B20204F
:1007960020535155454C4348205441494C20202074
:1007A60043544353532F44435320484F4C44204310
:1007B600524F535320425553592044454C415943B7
:1007C600524F5353204255535920484F4C442020F2
:1007D600204C54522053594E432042495420202045
:1007E600414456414E43454420204C4F434B202024
:1007F60020202020202020202020202020202020F3
:1008060020202020202020202020202020202020E2
:1008160020202020202020202020202020202020D2
:1008260020202020202020202020202020202020C2
:100836002020202020202020202020313D454E2031
:1008460020202020202020202020524154494F20C3
:1008560020202020202020202020303D434F5320E0
:1008660020202020202020202020313D504F5320C2
:10087600202020202020202020202031204D532001
:10088600202020202020202020203130204D5320E1
:10089600202020202020202020313030204D5320C1
:1008A60020202020202020202020202053454320C7
:1008B600202020202020202020313D534B4950204D
:1008C6002020202020202020202020202020202022
:1008D6002020202020202020202020202020202012
:1008E6005052494F52495459204C4556454C2020A8
:1008F6004C545220454E434F444520504F4C2020E7
:100906004C5452204445434F444520504F4C2020E0
:10091600205445535420494420434F444520204900
:10092600444C45204D45535341474520544D522094
:100936002020204152454120424954202020202099
:100946004D4153544552204F5220534C4156452059
:1009560044435320454E434F444520504F4C20209E
:10096600444353204445434F444520504F4C202098
:10097600434F5552544553592044454C4159202024
:10098600202048414E472054494D452020202043F1
:100996004152524945522044524F5020444C59200E
:1009A600204143434553532044454C41592020534D
:1009B600544154494F4E204944204D4F4445202030
:1009C600564F494345204F52204357494420202043
:1009D60020494420494E54455256414C202020205F
:1009E6002020435749442053504545442020202089
:1009F60043574944204652455155454E43592020B8
:100A06002043574944204D45535341474520202014
:100A16005455524E5F4F4E2044454C41592020209C
:100A26005455524E5F4F46462044454C415920206E
:100A360042454550204652455155454E4359205250
:100A4600455045415445522044495341424C452066
:100A56004155582052454C4159204D4F4445202080
:100A660043524F53532042555359204D4F4445202E
:100A76005245504541544552204741494E20202079
:100A86002054454C434F204741494E202020204EBC
:100A96004554574F524B2048414E4754494D4520E7
:100AA6002020202020202020204C4556454C202068
:100AB600202020202020202020303D4E4F524D2047
:100AC6002020202020202020202020434F44452085
:100AD6002020202020202020202020415245412077
:100AE60020202020202020303D4D415354455220C7
:100AF600202020202020202020202031204D53207F
:100B0600202020202020202020203130204D53205E
:100B1600202020202020202020313030204D53203E
:100B26002020202020202020203130205345432023
:100B36002020202020202020202031204D494E201A
:100B460020202020202020202020204D4F444520FA
:100B56002020202020202020303D564F494345208C
:100B660020202020202020202020204652455120D1
:100B76002020202020202020202020313D454E20EE
:100B860020414C41524D20434F554E5420202020A9
:100B9600524553544F524520434F554E5420202022
:100BA6002020494E54455256414C202020202020DA
:100BB6004E4554574F524B20434F44452020204921
:100BC6004E544552434F4E4E454354204D4F444E8E
:100BD6004554574F524B20494E414354495645823E
:100BE600010011022D15000182010111032D1500CE
:100BF6000182010211042D15000182010311052D48
:100C060015000178060411060119010182030A1173
:100C1600072E1500FF82030B11082E1500FF820315
:100C26000C11092E1500FF82030D110A2E1500FF67
:100C360082030E110B2E1500FF82030F110C2E15C9
:100C460000FF820310110D2E1500FF820311110EF5
:100C56002E1500FF820312110F2E1500FF820313BB
:100C660011102E1500FF82031411112E1500FF829C
:100C7600031511122E1500FF82031611132E1500EF
:100C8600FF82031711142E1500FF82031811152E6B
:100C96001500FF82011911162F15000182011A1184
:100CA600173015000182031B11182E1500FF820252
:100CB6001C11193115006382021D111A32150063C9
:100CC60082011E111B3015000182031F111C2E15F7
:100CD60000FF820220111D31150063820221111EC0
:100CE60032150063820222111F3315026382032329
:100CF6001120321501FF8203241121341502FF82CF
:100D060002251122331500638202261123321500B3
:100D160063820227112433150363820228112532C8
:100D26001500638203291126331500FA82012A1160
:100D3600273515000182012B11385415010982014E
:100D46002C11395515000182012D113A5515000156
:100D560082032E113B561501FA82032F113C5C15B6
:100D660000FF820130113D57150001820131113E0D
:100D760058150001820132113F55160001820133D8
:100D860011405515000182023411415A1500638243
:100D9600023511425B15006382023611435A150073
:100DA6006382023711445A15006382013811455E89
:100DB60015000182013911465F15000182023A11C0
:100DC600475D15006382023B114859150463820290
:100DD6003C114960150114BE0A3D114A5611000026
:100DE600820247114B5A150063820248114D601565
:100DF6000114820149114E5E15000282014A114F0B
:100E06006115000182014B11505E15000482014CF0
:100E160011515415010982014D11525415010982CF
:100E2600024E11533415006382014F116201150001
:100E36000982015011630115000982025111645D96
:100E4600150163C803521165011501018201541190
:100E5600665E1500028203551167341500FF010115
:100E66000200000200000200000000000001010173
:100E76003132333435361432320532FFFFFF191959
:100E8600196464C8FF000180000A0180000A1E1A66
:100E9600B400001E1E1E0001000002010001000039
:100EA6000A1E630A000100050520202020202020BC
:100EB6002020200A050000000101140000010000A6
:020EC60000002A
:10973D008B758A7689777F01127D7BE49000E7F047
:10974D009000E7E0FFC39410501AAB75AA76A97785
:10975D008F827583001284ABFF127D4C9000E7E081
:05976D0004F080DC2285
:109772008B758A7689777F11127D7BE49000E7F002
:109782009000E7E0FFC39410501AAB75AA76A97750
:109792008F827583001284ABFF127D4C9000E7E04C
:0597A20004F080DC2250
:104ABF00E49001A8F0A3F09001AAF09000EBF0A30E
:104ACF00F09000ECE02400F582E43404F583E4F088
:104ADF009000ECE004F070069000EBE004F0900022
:104AEF00EBE07004A3E0648070D7E49000E7F090EF
:104AFF0000E7E0FFC394024003024B90EF900E6477
:104B0F0093FF9001AAE0FE04F074002EF582E434C6
:104B1F0004F583EFF09001AAE06480705B9001A828
:104B2F00E0FEA3E07807C333CE33CED8F9FF7C0481
:104B3F007D001273D3E49000EBF0A3F09000ECE053
:104B4F002400F582E43404F583E4F09000ECE004F3
:104B5F00F070069000EBE004F09000EBE07004A31F
:104B6F00E0648070D7E49001AAF09001A9E004F00E
:104B7F0070069001A8E004F09000E7E004F0024A0C
:104B8F00FEE49000EAF0E49000E8F0A3F0E4900077
:104B9F00E7F09000E7E0FFC394034003024C33EFCC
:104BAF00900E6693FF9001AAE0FE04F074002EF5BC
:104BBF0082E43404F583EFF09001AAE06480705B27
:104BCF009001A8E0FEA3E07807C333CE33CED8F927
:104BDF00FF7C047D001273D3E49000EBF0A3F09000
:104BEF0000ECE02400F582E43404F583E4F0900057
:104BFF00ECE004F070069000EBE004F09000EBE0C6
:104C0F007004A3E0648070D7E49001AAF09001A92A
:104C1F00E004F070069001A8E004F09000E7E004D3
:104C2F00F0024BA19000E9E004F070069000E8E07C
:104C3F0004F0C39000E9E094339000E8E094005052
:104C4F0003024B9C9000EAE004F0E0C3941450037D
:104C5F00024B95E49000EAF0E49000E8F0A3F0E452
:104C6F009000E7F09000E7E0FFC394034003024D8C
:104C7F0005EF900E6993FF9001AAE0FE04F0740017
:104C8F002EF582E43404F583EFF09001AAE06480FE
:104C9F00705B9001A8E0FEA3E07807C333CE33CE5C
:104CAF00D8F9FF7C047D001273D3E49000EBF0A3DE
:104CBF00F09000ECE02400F582E43404F583E4F096
:104CCF009000ECE004F070069000EBE004F0900030
:104CDF00EBE07004A3E0648070D7E49001AAF09039
:104CEF0001A9E004F070069001A8E004F09000E73D
:104CFF00E004F0024C739000E9E004F070069000BD
:104D0F00E8E004F0C39000E9E094709000E8E094CC
:104D1F00005003024C6E9000EAE004F0E0C39414DC
:104D2F005003024C67E49000E8F0A3F0E49000E732
:104D3F00F09000E7E0FFC394034003024DD2EF90E1
:104D4F000E6C93FF9001AAE0FE04F074002EF58222
:104D5F00E43404F583EFF09001AAE06480705B9077
:104D6F0001A8E0FEA3E07807C333CE33CED8F9FF16
:104D7F007C047D001273D3E49000EBF0A3F090005D
:104D8F00ECE02400F582E43404F583E4F09000ECC9
:104D9F00E004F070069000EBE004F09000EBE070A0
:104DAF0004A3E0648070D7E49001AAF09001A9E019
:104DBF0004F070069001A8E004F09000E7E004F022
:104DCF00024D409000E9E004F070069000E8E00426
:104DDF00F0C39000E9E094889000E8E0941350034A
:104DEF00024D3B8000E49000E8F0A3F0E49000E770
:104DFF00F09000E7E0FFC394564003024E92EF900D
:104E0F000E7293FF9001AAE0FE04F074002EF5825B
:104E1F00E43404F583EFF09001AAE06480705B90B6
:104E2F0001A8E0FEA3E07807C333CE33CED8F9FF55
:104E3F007C047D001273D3E49000EBF0A3F090009C
:104E4F00ECE02400F582E43404F583E4F09000EC08
:104E5F00E004F070069000EBE004F09000EBE070DF
:104E6F0004A3E0648070D7E49001AAF09001A9E058
:104E7F0004F070069001A8E004F09000E7E004F061
:104E8F00024E009000E9E004F070069000E8E004A4
:104E9F00F0C39000E9E094149000E8E09400500310
:104EAF00024DFB9001A8E0FEA3E07807C333CE3399
:104EBF00CED8F9FF7C047D001273D3127D95027D4D
:014ECF00A43E
:109A7000E4900059F0A3F0FFFE12737C90005BEFBE
:029A8000F022D2
:1086FE0075530175540075556AE49001F6F0A3F0B8
:10870E009001F6E0FAA3E0FBC39456EA94005040C1
:10871E0090005BE075F056A42478FFE5F03460CF4E
:10872E002BCF3AFE900059F0A3EFF012737CAB53AF
:10873E000555E555AA547002055414F9EF1284D864
:10874E009001F7E004F070B89001F6E004F080B00C
:10875E0090009BE07004D2588002C258900097E0BF
:10876E0024FF924F900096E024FF924490009DE0EB
:10877E0024FF924E90009CE024FF924590007CE0F6
:02878E00F52DC7
:0187900022C6
:108F8F007553017554007555BFE49001F6F0A3F0C9
:108F9F009001F6E0FEA3E0FFC39414EE9400503B63
:108FAF007C007D561284EAEF24F9FFEE3460FE90C8
:108FBF000059F0A3EFF012737CAB530555E555AA9A
:108FCF00547002055414F9EF1284D89001F7E0049D
:0B8FDF00F070BD9001F6E004F080B5DA
:018FEA002264
:108FEB007553017554007555D3E49001F6F0A3F059
:108FFB009001F6E0FEA3E0FFC39414EE9400503B07
:10900B007C007D561284EAEF24FEFFEE3460FE9066
:10901B000059F0A3EFF012737CAB530555E555AA3D
:10902B00547002055414F9EF1284D89001F7E00440
:0B903B00F070BD9001F6E004F080B57D
:019046002207
:108BBF008F75E49000E7F09000E7E0FBC39403505B
:108BCF003E90005BE075F099A42469FDE5F034FF59
:108BDF00FCE57575F003A42DFFE5F03CFEEB7C0082
:108BEF002FFFEC3EFE12737C9000E7E02461F582CC
:108BFF00E43400F583EFF09000E7E004F080B890E4
:108C0F000061E0FE540190005CF0EE540290005DB4
:108C1F00F0900061E0540490005EF0EE5408900074
:0D8C2F005FF0900061E05410900060F022B2
:1089BC008F75E49000E7F09000E7E0FBC394035060
:1089CC004490005BE0FF7E007C017D501284EAEF56
:1089DC0024A6FDEE340AFCE57575F003A42DFFE525
:1089EC00F03CFEEB7C002FFFEC3EFE12737C900003
:1089FC00E7E02461F582E43400F583EFF09000E7C2
:108A0C00E004F080B2900061E0FE540190005CF054
:108A1C00EE540290005DF0900061E0540490005E12
:108A2C00F0EE540890005FF0900061E0541090005C
:038A3C0060F022C5
:0685D3008F758C768D7798
:1085D900E49001F6F0A3F0E57724FFFFE57634FF98
:1085E900FE7C007D031284EAAA06AB07AE75E57529
:1085F90025E0CE75F0EEA4FFE5F02EFEEF2448FF4E
:10860900EE3423CF2BCF3AFE9001F7E02FFF9001F4
:10861900F6E03EFE12737C9001F7E02461F582E4F6
:108629003400F583EFF09001F7E004F07006900153
:10863900F6E004F0C39001F7E094039001F6E094AA
:10864900004094900061E0FE5401900067F0EE5400
:0F86590002900068F0900061E05404900069F016
:0186680022EF
:10994A002020202020534C41564520202020202032
:10995A0020202020204D41535445522020202020F1
:0E9AC300127CA9127D95127DA47F01027D7B8D
:1097A7009000037414F0127D95900003E070FA9016
:1097B700009BE07BFF60067A99794A80047A997961
:1097C7005A1297729000037414F0127D959000035B
:0497D700E070FA2222
:1076EF00C0D0C0E0C0F0C000A88475840FE5585426
:1076FF0007B4000D85E8F0A2F09220A2F19221804C
:10770F0076B4010D85E8F0A2F09222A2F1922380C7
:10771F0066B4020D85E8F0A2F09224A2F1922580C2
:10772F0056B4030D85E8F0A2F09226A2F1922780BD
:10773F0046B4040D85E8F0A2F09218A2F1921980D8
:10774F0036B4050D85E8F0A2F0921AA2F1921B80D3
:10775F0026B4060D85E8F0A2F0921CA2F1921D80CE
:10776F001685E8F0A2F0921EA2F1921F7558FF85C0
:10777F00231E85241FD260055875590A8884D000AE
:10778F00D0F0D0E0D0D032205F0122D2B7E55A54EA
:10779F0007B4000AA22F92F7A22E92F6805EB401D0
:1077AF000AA22D92F7A22C92F68051B4020AA22BB4
:1077BF0092F7A22A92F68044B4030AA22992F7A262
:1077CF002892F68037B4040AA23792F7A23692F6BF
:1077DF00802AB4050AA23592F7A23492F6801DB41E
:1077EF00060AA23392F7A23292F68010B40721A2B2
:1077FF003192F7A23092F6C25F755AFF055A75841F
:10780F000F85E8E0A2F692E6A2F792E7F5E8C2B795
:01781F002246
:108F2F009001D2E0FFEF1285128F5D008F61018FEC
:108F3F0065028F69038F6D048F71058F75068F79A9
:108F4F00078F7D088F81098F850A00008F89128D09
:108F5F002D221286692212914B22128C3C22127FF3
:108F6F00B2221283E222127DB32212957422129240
:108F7F004322125EC42212609D229001D2E4F0229D
:108D2D003061669001D3E4F0C261E5561285128D73
:108D3D005B478D62488D69498D704A8D774B8D7E6D
:108D4D004C8D854D8D8C4E8D904F00008D969001E4
:108D5D00D27401F0229001D27402F0229001D274EB
:108D6D0003F0229001D27404F0229001D27405F028
:108D7D00229001D27406F0229001D27407F02212D3
:0A8D8D009A0C229001D27408F02223
:108669009001D3E0FFEF70189001DA7401F09001E6
:10867900DB7401F09001D27409F09001D3E4F02287
:108689009001D3E0FFEFB401189001DA7401F09082
:1086990001DB7402F09001D2740AF09001D3E4F086
:1086A900229001D3E0FFEF640270499001D8E4F011
:1086B900A3E4F09001D8E475F0011284FCAFF0FE58
:1086C900EF4E60269001D4E475F0011284FCAFF0FE
:1086D900FE9001D8E0FCA3E0FD74002DF58274083A
:1086E9003CF583E0FD12733B80C97F01120086903F
:0586F90001D2E4F022B3
:10914B009001D3E0FFEF70189001DA7402F09001F8
:10915B00DB7401F09001D27409F09001D3E4F0229A
:10916B009001D3E0FFEFB401189001DA7402F09094
:10917B0001DB7402F09001D2740AF09001D3E4F099
:10918B00229001D3E0FFEFB4020A7F011200869018
:05919B0001D2E4F02206
:108C3C009001D3E0FFEF70189001DA7403F090010B
:108C4C00DB7401F09001D27409F09001D3E4F022AE
:108C5C009001D3E0FFEFB401189001DA7403F090A7
:108C6C0001DB7402F09001D27409F09001D3E4F0AE
:108C7C00229001D3E0FFEFB4021C205F2F9001D4AF
:108C8C00E0FEA3E0FF9001C2EEF0A3EFF0D25F9004
:108C9C0001D3E004F0229001D3E0FFEFB4030D20E8
:0D8CAC005F0A7F011200869001D2E4F022E1
:107FB2009001D3E0FFEF70189001DA7404F09001A1
:107FC200DB7401F09001D27409F09001D3E4F02245
:107FD2009001D3E0FFEF640170749001D6E0FEA33C
:107FE200E0FF9001D8EEF0A3EFF09001E0E4F0A3FF
:107FF200E4F09001D8E4F0A3E4F09001D8E475F045
:10800200011284FCAFF0FEEF4E602B9001D4E475B8
:10801200F0011284FCAFF0FE12737C9001E0E47573
:10802200F0011284FCADF0FC74002DF58274083C62
:10803200F583EFF080C4900800E0FF120086900103
:10804200E0E4F0A37401F09001D3E004F022900187
:10805200D3E0FFEF6402703F30624D9001E0E475BF
:10806200F0011284FCAFF0FE74002FF58274083E1A
:10807200F583E0FF1200869001D6E0FEA3E0FF90B8
:1080820001E0E0FCA3E0FDC3ED9FEC9E5002222242
:108092009001D3E004F0229001D3E0FFEFB4030893
:0980A2003062059001D2E4F022E5
:1083E2009001D3E0FFEF70189001DA7405F090016C
:1083F200DB7401F09001D27409F09001D3E4F02211
:108402009001D3E0FFEFB4012C9001D6E0FEA3E08F
:10841200FF128B40900800E0FF1200869001D67494
:1084220004F0A3E4F09001E0E4F0A37401F0900101
:10843200D3E004F0229001D3E0FFEF6402703F30FA
:10844200624D9001E0E475F0011284FCAFF0FE741D
:10845200002FF58274083EF583E0FF12008690013A
:10846200D6E0FEA3E0FF9001E0E0FCA3E0FDC3ED57
:108472009FEC9E500222229001D3E004F022900150
:10848200D3E0FFEFB403083062059001D2E4F0229A
:107DB3009001D3E0FFEF70189001DA7406F09001A0
:107DC300DB7401F09001D27409F09001D3E4F02246
:107DD3009001D3E0FFEFB401289001C27430F0A307
:107DE300E4F09001D4E0FEA3E0FF9001C4EEF0A321
:107DF300EFF09001BE7402F0D25F9001D3E004F083
:107E0300229001D3E0FFEFB4020D305F03027EB492
:107E13009001D3E004F0229001D3E0FFEFB4030D0F
:107E2300205E03027EB49001D3E004F0229001D3DC
:107E3300E0FFEFB40421900800E0FF1200869001F8
:107E4300D67404F0A3E4F09001E0E4F0A37401F02D
:107E53009001D3E004F0229001D3E0FFEF640570BA
:107E63003F30624D9001E0E475F0011284FCAFF005
:107E7300FE74002FF58274083EF583E0FF1200863E
:107E83009001D6E0FEA3E0FF9001E0E0FCA3E0FD5B
:107E9300C3ED9FEC9E500222229001D3E004F02216
:107EA3009001D3E0FFEFB406083062059001D2E4FD
:027EB300F022BB
:109574009001D3E0FFEF7011C2619001D47402F046
:10958400A3E4F09001D3E004F09001D3E0FFEFB442
:10959400011A205D179001D4E0FEA3E0FF9001C200
:0D95A400EEF0A3EFF0D25D9001D2E4F022D2
:109243009001D3E0FFEF7024306144C2619001D4F8
:109253007401F0A3E4F0AF567E009001D5E02FF047
:109263009001D4E03EF09001D3E004F09001D3E00C
:10927300FFEFB4011A205D179001D4E0FEA3E0FFD5
:109283009001C2EEF0A3EFF0D25D9001D2E4F022A0
:105EC40020610302609CC2619001D3E0FFEF701671
:105ED400AF561288AF7E009001D4EEF0A3EFF0909D
:105EE40001D3E004F0229001D3E0FFEFB401389035
:105EF40001D4E0FEA3E0FFEFC4F8540FC868FFEE3E
:105F0400C454F048FE9001D4EEF0A3EFF0AF561263
:105F140088AF7E009001D5E02FF09001D4E03EF0F0
:105F24009001D3E004F0229001D3E0FFEFB40238F3
:105F34009001D4E0FEA3E0FFEFC4F8540FC868FF5B
:105F4400EEC454F048FE9001D4EEF0A3EFF0AF5647
:105F54001288AF7E009001D5E02FF09001D4E03E8E
:105F6400F09001D3E004F0229001D3E0FFEFB403FA
:105F7400389001D4E0FEA3E0FFEFC4F8540FC868E2
:105F8400FFEEC454F048FE9001D4EEF0A3EFF0AF5E
:105F9400561288AF7E009001D5E02FF09001D4E036
:105FA4003EF09001D3E004F0229001D3E0FFEFB47F
:105FB4000416AF561288AF7E009001D6EEF0A3EF20
:105FC400F09001D3E004F0229001D3E0FFEFB40598
:105FD400389001D6E0FEA3E0FFEFC4F8540FC86880
:105FE400FFEEC454F048FE9001D6EEF0A3EFF0AFFC
:105FF400561288AF7E009001D7E02FF09001D6E0D2
:106004003EF09001D3E004F0229001D3E0FFEFB41E
:1060140006389001D6E0FEA3E0FFEFC4F8540FC8A1
:1060240068FFEEC454F048FE9001D6EEF0A3EFF002
:10603400AF561288AF7E009001D7E02FF09001D6C2
:10604400E03EF09001D3E004F0229001D3E0FFEFB2
:10605400B407459001D6E0FEA3E0FFEFC4F8540F67
:10606400C868FFEEC454F048FE9001D6EEF0A3EFEA
:10607400F0AF561288AF7E009001D7E02FF0900168
:10608400D6E03EF09001DBE0FF9001D3EFF0900109
:09609400DAE0FF9001D2EFF022E6
:10609D009001D3E0FFEF70279001E0E4F0A3E4F06E
:1060AD009001D6E0FEA3E0FF9001D8EEF0A3EFF053
:1060BD009001DEE4F0A3E4F09001D3E004F022209F
:1060CD0061030262739001D3E0FFEFB4010EAF568E
:1060DD001288AF8F7C9001D3E004F0229001D3E0C1
:1060ED00FFEF6402706CE57CC454F0F57CAF561282
:1060FD0088AFEF257CF57C9001E0E0FEA3E0FF7416
:10610D00002FF58274083EF583E57CF0AF7C7E00B0
:10611D009001DFE02FF09001DEE03EF09001E1E034
:10612D0004F070069001E0E004F09001D9E024FF46
:10613D00F09001D8E034FFF09001D8E0FEA3E0FF2D
:10614D00EF4E60079001D37401F0229001D3E0046B
:10615D00F0229001D3E0FFEFB40316AF561288AFD3
:10616D007E009001DCEEF0A3EFF09001D3E004F09F
:10617D00229001D3E0FFEFB404389001DCE0FEA3E0
:10618D00E0FFEFC4F8540FC868FFEEC454F048FEAA
:10619D009001DCEEF0A3EFF0AF561288AF7E0090C9
:1061AD0001DDE02FF09001DCE03EF09001D3E00442
:1061BD00F0229001D3E0FFEFB405389001DCE0FE52
:1061CD00A3E0FFEFC4F8540FC868FFEEC454F048C5
:1061DD00FE9001DCEEF0A3EFF0AF561288AF7E001B
:1061ED009001DDE02FF09001DCE03EF09001D3E076
:1061FD0004F0229001D3E0FFEF640670699001DC9A
:10620D00E0FEA3E0FFEFC4F8540FC868FFEEC454DE
:10621D00F048FE9001DCEEF0A3EFF0AF561288AF20
:10622D007E009001DDE02FF09001DCE03EF090016A
:10623D00DCE0FEA3E0FF9001DEE0FCA3E0FDEDB5A8
:10624D00071AECB506169001DAE0FF9001D2EFF0D7
:10625D009001DBE0FF9001D3EFF022227F021200CC
:07626D00869001D2E4F0224B
:1088AF008F7AE57AB430037F0022E57AB431037F03
:1088BF000122E57AB432037F0222E57AB433037FD3
:1088CF000322E57AB434037F0422E57AB435037FBB
:1088DF000522E57AB436037F0622E57AB437037FA3
:1088EF000722E57AB438037F0822E57AB439037F8B
:1088FF000922E57AB441037F0A22E57AB442037F65
:10890F000B22E57AB443037F0C22E57AB444037F4C
:10891F000D22E57AB445037F0E22E57AB446037F34
:07892F000F22D2637F00223A
:0B0086008F7B758400857B99D262227D
:109A0C00C2B5900003741EF0900003E0FFEF6004F9
:079A1C00C2B580F4D2B522AF
:105CC40000000000000004000000080000000C00B8
:105CD40000001000000014000000180000001C0068
:105CE40000002000000024000000280000002C0018
:105CF40000003000000034000000380000003C00C8
:105D040000004000000044000000480000004C0077
:105D140000005000000054000000580000005C0027
:105D240000006000000064000000680000006C00D7
:105D340000007000000074000000780000007C0087
:105D440000108000001084000010880000108C00F7
:105D540000109000001094000010980000109C00A7
:105D64000010A0000010A4000010A8000010AC0057
:105D74000010B0000010B4000010B8000010BC0007
:105D84000010C0000010C4000010C8000010CC00B7
:105D94000010D0000010D4000010D8000010DC0067
:105DA4000010E0000010E4000010E8000010EC0017
:105DB4000010F0000010F4000010F8000010FC00C7
:105DC40000218000002184000021880000218C0033
:105DD40000219000002194000021980000219C00E3
:105DE4000021A0000021A4000021A8000021AC0093
:105DF4000021B0000021B4000021B8000021BC0043
:105E04000021C0000021C4000021C8000021CC00F2
:105E14000021D0000021D4000021D8000021DC00A2
:105E24000021E0000021E4000021E8000021EC0052
:105E34000021F0000021F4000021F8000021FC0002
:105E440000318000003184000031880000318C0072
:105E540000319000003194000031980000319C0022
:105E64000031A0000031A4000031A8000031AC00D2
:105E74000031B0000031B4000031B8000031BC0082
:105E84000031C0000031C4000031C8000031CC0032
:105E94000031D0000031D4000031D8000031DC00E2
:105EA4000031E0000031E4000031E8000031EC0092
:105EB4000031F0000031F4000031F8000031FC0042
:10422B009001ADE0FFEF70769001BFE0FFEFD3940C
:10423B0003400302468F20600302468FC260900149
:10424B00BCE51EF0A3E51FF09001BCE0FEA3E0FF70
:10425B00EE541FFE9001B6EEF0A3EFF09001BCE020
:10426B00FEA3E0FFEEC4135407FF7E009001BCEEEB
:10427B00F0A3EFF09001BDE0FF9001AFEFF09001E4
:10428B00AEE4F09001BCE0FEA3E0FFEF4E7004D271
:10429B005E22229001BDE0FF9001ADEFF022900174
:1042AB00ADE0FFEFB4011A20600302468F9001B816
:1042BB00E51EF0A3E51FF0C260D25E9001ADE4F005
:1042CB00229001ADE0FFEF640270402060030246D4
:1042DB008FC2609001AEE0FFEF70119001B8E51E48
:1042EB00F0A3E51FF09001AEE004F0229001AEE0E8
:1042FB00FFEF6401600302468F9001BAE51EF0A345
:10430B00E51FF0D25E9001ADE4F0229001ADE0FF2D
:10431B00EF6403600302443C20600302468F90016C
:10432B00A7740AF0C2609001AEE0FFEF7029900114
:10433B00B8E51EF0A3E51FF09001B4E4F0A3E4F0A0
:10434B009001B0E4F0A3E4F09001B2E4F0A3E4F048
:10435B009001AEE004F0229001AEE0FFEF6401703B
:10436B00799001BCE51EF0A3E51FF09001BCE0FEC7
:10437B00A3E0FF9001B1E02FF09001B0E03EF09090
:10438B0001BCE0FCA3E0FD9001B2E475F0011284E6
:10439B00FCAFF0FEEF25E0FFEE33FE74002FF5824D
:1043AB0074043EF583ECF0A3EDF09001B5E004F05E
:1043BB0070069001B4E004F09001B6E0FEA3E0FFBC
:1043CB009001B4E0FCA3E0FDED6F7002EC6E6003B6
:1043DB0002468F9001AE7402F0229001AEE0FFEF27
:1043EB006402600302468F9001BAE51EF0A3E51F3D
:1043FB00F09001ADE4F09001B0E0FEA3E0FF90017E
:10440B00BAE0FCA3E0FDEDB5071FECB5061B900170
:10441B00B6E0FEA3E0FF9001B8E0FCA3E0FD129232
:10442B00937F007E90129A4B227F017E90129A4BC3
:10443B00229001ADE0FFEF6404600302456D206044
:10444B000302468F9001A7740AF0C2609001AEE0A0
:10445B00FFEF70299001B8E51EF0A3E51FF0900166
:10446B00B4E4F0A3E4F09001B0E4F0A3E4F0900125
:10447B00B2E4F0A3E4F09001AEE004F0229001AEC0
:10448B00E0FFEF640170739001BCE51EF0A3E51F24
:10449B00F09001BCE0FEA3E0FF9001B1E02FF090A3
:1044AB0001B0E03EF09001BCE0FCA3E0FD9001B256
:1044BB00E475F0011284FCAFF0FEEF25E0FFEE3364
:1044CB00FE74002FF58274043EF583ECF0A3EDF03F
:1044DB009001B5E004F070069001B4E004F0900197
:1044EB00B4E0FEA3E0FFEF64007003EE6402600330
:1044FB0002468F9001AEE004F0229001AEE0FFEF98
:10450B006402600302468F755B559001BAE51EF09D
:10451B00A3E51FF09001B0E0FEA3E0FF9001BAE02D
:10452B00FCA3E0FDEDB50727ECB506239001B6E043
:10453B00FEA3E0FF127EB57F007E90129A4B900196
:10454B00B8E0FEA3E0FFEF4E6012755CAA800D751C
:10455B005B00755C007F017E90129A4B9001ADE47D
:10456B00F0229001ADE0FFEF6405600302467A2074
:10457B00600302468F9001A7740AF0C2609001AEEF
:10458B00E0FFEF70299001B8E51EF0A3E51FF09056
:10459B0001B4E4F0A3E4F09001B0E4F0A3E4F090F4
:1045AB0001B2E4F0A3E4F09001AEE004F02290013C
:1045BB00AEE0FFEF640170769001BCE51EF0A3E561
:1045CB001FF09001BCE0FEA3E0FF9001B1E02FF0E3
:1045DB009001B0E03EF09001BCE0FCA3E0FD900147
:1045EB00B2E475F0011284FCAFF0FEEF25E0FFEEB4
:1045FB0033FE74002FF58274043EF583ECF0A3EDCB
:10460B00F09001B5E004F070069001B4E004F09076
:10461B0001B6E0FEA3E0FF9001B4E0FCA3E0FDEDEA
:10462B006F7002EC6E705D9001AEE004F0229001B1
:10463B00AEE0FFEF6402704C9001BAE51EF0A3E50B
:10464B001FF09001ADE4F09001B0E0FEA3E0FF900D
:10465B0001BAE0FCA3E0FDEDB5070CECB506087F55
:10466B00007E90129A4B227F017E90129A4B2290E1
:10467B0001ADE0FFEFD39405400A9001ADE4F0905B
:05468B0001AEE4F02285
:1032DD009001BFE0FFEF702A9001ADE0FFEFD394B6
:1032ED00024003023844305F03023844205D03027C
:1032FD0038449001BEE0FF9001BFEFF09001C0E4B3
:10330D00F0229001BFE0FFEFB401179001C2E0FE83
:10331D00A3E0FFEE4420FE129A4BC25D9001BFE484
:10332D00F0229001BFE0FFEF640270489001C0E011
:10333D00FFEF7019205F169001C2E0FEA3E0FFEED3
:10334D004440FE129A4B9001C0E004F0229001C05F
:10335D00E0FFEFB4011E305F030238449001C4E07A
:10336D00FEA3E0FF129A4BC25D9001BFE4F0900105
:10337D00C0E4F0229001BFE0FFEF6403706C900198
:10338D00C0E0FFEF701C305F030238449001C2E0D3
:10339D00FEA3E0FFEE4460FE129A4B9001C0E004E4
:1033AD00F0229001C0E0FFEFB40118305F03023846
:1033BD00449001C4E0FEA3E0FF129A4B9001C0E0DF
:1033CD0004F0229001C0E0FFEFB4021E305F030253
:1033DD0038449001C6E0FEA3E0FF129A4BC25D9007
:1033ED0001BFE4F09001C0E4F0229001BFE0FFEFD7
:1033FD006404600302358D9001C0E0FFEF703390DF
:10340D0001C2E0FEA3E0FF9001C4E0FCA3E0FD12C9
:10341D0091A09001CAE4F0A3E4F09001CCE4F0A3F4
:10342D007480F09001C8E4F0A3E4F09001C0E004D2
:10343D00F0229001C0E0FFEFB4011C305F030238B1
:10344D00449001C2E0FEA3E0FFEE4480FE129A4BD1
:10345D009001C0E004F0229001C0E0FFEFB402182B
:10346D00305F030238449001C4E0FEA3E0FF129ADE
:10347D004B9001C0E004F0229001C0E0FFEF640327
:10348D007063305F030238449001C8E475F0011297
:10349D0084FCAFF0FEEF25E0FFEE33FE74002FF558
:1034AD008274043EF583E0F570A3E0F571AF71AE63
:1034BD0070129A4B9001CBE02571F09001CAE03566
:1034CD0070F09001CDE024FFF09001CCE034FFF0DE
:1034DD009001CCE0FEA3E0FFEF4E600222229001AE
:1034ED00C0E004F0229001C0E0FFEFB4041E305F95
:1034FD00030238449001CAE0FEA3E0FF129A4B90FC
:10350D0001C17464F09001C0E004F0229001C0E0AC
:10351D00FFEF6405706A9001C1E0FFEF7019900133
:10352D00CFE004F070069001CEE004F09001BFE40E
:10353D00F09001C0E4F022306046C260851E7285B5
:10354D001F739001C0E4F0E573B40011E572B490FF
:10355D000C9001BFE4F09001C0E4F0C25DE573642E
:10356D00017004E572649060030238449001C0E478
:10357D00F09001CFE004F070069001CEE004F0224F
:10358D009001BFE0FFEF640560030238449001C075
:10359D00E0FFEF702B9001CAE4F0A3E4F09001CCB2
:1035AD007402F0A3E4F09001C8E4F0A3E4F09001FC
:1035BD00C2E0FEA3E0FF128B409001C0E004F022B8
:1035CD009001C0E0FFEFB4011C305F03023844905E
:1035DD0001C2E0FEA3E0FFEE44A0FE129A4B900163
:1035ED00C0E004F0229001C0E0FFEF640270633090
:1035FD005F030238449001C8E475F0011284FCAFFA
:10360D00F0FEEF25E0FFEE33FE74002FF58274041B
:10361D003EF583E0F570A3E0F571AF71AE70129ACF
:10362D004B9001CBE02571F09001CAE03570F09020
:10363D0001CDE024FFF09001CCE034FFF09001CCFF
:10364D00E0FEA3E0FFEF4E600222229001C0E004F5
:10365D00F0229001C0E0FFEFB4031E305F0302388B
:10366D00449001CAE0FEA3E0FF129A4B9001C17491
:10367D0064F09001C0E004F0229001C0E0FFEF641F
:10368D000470659001C1E0FFEF70149001CFE0046C
:10369D00F070069001CEE004F09001C0E4F022300D
:1036AD006046C260851E72851F739001C0E4F0E50F
:1036BD0073B40011E572B4900C9001BFE4F0900169
:1036CD00C0E4F0C25DE57364017004E5726490605E
:1036DD00030238449001CFE004F070069001CEE073
:1036ED0004F09001C0E4F0229001C0E0FFEF7020E3
:1036FD009001CAE4F0A3E4F09001CC7402F0A3E4CD
:10370D00F09001C8E4F0A3E4F09001C0E004F022D1
:10371D009001C0E0FFEFB4011C305F03023844900C
:10372D0001C2E0FEA3E0FFEE44C0FE129A4B9001F1
:10373D00C0E004F0229001C0E0FFEF64027063303E
:10374D005F030238449001C8E475F0011284FCAFA8
:10375D00F0FEEF25E0FFEE33FE74002FF5827404CA
:10376D003EF583E0F570A3E0F571AF71AE70129A7E
:10377D004B9001CBE02571F09001CAE03570F090CF
:10378D0001CDE024FFF09001CCE034FFF09001CCAE
:10379D00E0FEA3E0FFEF4E600222229001C0E004A4
:1037AD00F0229001C0E0FFEFB4031E305F0302383A
:1037BD00449001CAE0FEA3E0FF129A4B9001C0E0D5
:1037CD0004F09001C17464F0229001C0E0FFEF6439
:1037DD000470649001C1E0FFEF70199001CFE00417
:1037ED00F070069001CEE004F09001C0E4F090017D
:1037FD00BFE4F022306040C260851E72851F739059
:10380D0001C0E4F0E573B40011E572B4900C9001C1
:10381D00BFE4F09001C0E4F0C25DE573B40118E5BA
:10382D0072B490139001C0E4F09001CFE004F070F9
:07383D00069001CEE004F04B
:013844002261
:047EB5008E0F8F108D
:107EB900D3E510947DE50F940040047F0180027F93
:107EC90000C3E510943FE50F940050047E01800241
:107ED9007E00EE4FFFEF6003027FB1E510AE0F7831
:107EE90002C333CE33CED8F9FF74C62FF582745C42
:107EF9003EF583E493F511740193F512E510AE0F85
:107F09007802C333CE33CED8F9FF74C42FF5827407
:107F19005C3EF583E493FE740193FF8F179001ADE6
:107F2900E0FFEF6405FF9001E8EFF09001AEE0FF9C
:107F3900EF6401FF9001E9EFF0AD12AC11AF171238
:107F490095379001ADE0FFEF6405FF9001E8EFF090
:107F59009001AEE0FFEF6403FF9001E9EFF07515C2
:107F690000751600C3E51594045033AE15AF1674A9
:107F7900002FF58274043EF583E0FF7E008E138F97
:107F890014AB14AD12AC11AF171293690512E512B7
:107F9900700205110516E5167002051580C69001D7
:087FA900E8E4F09001E9E4F0C6
:017FB10022AD
:089293008E648F658C668D6707
:10929B00756800756900E56525E0FFE56433FEC37D
:1092AB00E5699FE5689E50290567E567AE66700224
:1092BB00056614FFAC68AD6974002DF58274043C2F
:1092CB00F583E0FD12733B0569E569700205688063
:0192DB00C5CD
:0192DC00226F
:048B40008E5D8F5E59
:108B4400E55EAE5D7802C333CE33CED8F9FF74C68A
:108B54002FF582745C3EF583E493F55F740193F51D
:108B640060E55EAE5D7802C333CE33CED8F9FF74D0
:108B7400C42FF582745C3EF583E493FE740193FF85
:108B84008F63756100756200C3E5619404502BAD79
:108B940060AC5FAF6312992AAC61AD6274002DF5CD
:108BA4008274043CF583EFF00560E5607002055FB4
:0A8BB4000562E5627002056180CEE3
:018BBE002294
:0891A0008E6A8F6B8C6C8D6DE3
:1091A800756E00756F00E56B2401FFE56A3400FEFB
:1091B800EF25E0FFEE33FEC3E56F9FE56E9E502975
:1091C800056DE56DAE6C7002056C14FF12737CAC16
:1091D8006EAD6F74002DF58274043CF583EFF005D5
:0991E8006FE56F7002056E80BD99
:0191F100225B
:109A4B008E188F19205FFD851825851926755A00EC
:039A5B00D25F22B5
:1075B400205E030276EE9001AFE0FFEF60030276F7
:1075C4007BC25E9001B6E0FEA3E0FFEFB4FF0BEEDA
:1075D400B41F0775840075EF03229001B6E0FEA383
:1075E400E0FFEEFF7E008F789001B7E0FFEF54FFDD
:1075F400F579E578700B7FFF8F799001E57401F0E0
:1076040022E578B41516C3E579648094B3500D90DF
:1076140001E27401F09001E4E579F022E578B41612
:1076240016C3E579648094F2500D9001E27402F07F
:107634009001E4E579F022D3E578648094804037C2
:10764400C3E57864809495502ED3E5796480948062
:107654004025AF79EF3395E0FEC3EF94FBEE6480F1
:10766400948050139001E27403F09001E3E578F004
:107674009001E4E579F0229001AFE0FFEF6402703D
:10768400699001B6E0FEA3E0FFEF64014E702B9019
:1076940001BFE0FFEF70F89001C2E4F0A3747FF043
:1076A4009001BAE0FEA3E0FF9001C4EEF0A3EFF076
:1076B4009001BE7404F0D25DC25E9001B6E0FEA3F8
:1076C400E0FFEF64024E70229001BFE0FFEF70F81C
:1076D4009001BAE0FEA3E0FF9001C2EEF0A3EFF048
:0A76E4009001BE7405F0D25DC25E95
:0176EE002279
:10FC0000C2AF12FCD812FD10E4F550F551E42551B5
:10FC1000FFE5503480FE12FCB6AD07AF51AE501276
:10FC2000FC5F0551E55170020550C3E550948040DA
:10FC3000DC755080755100AF51AE5012FCC7AD0756
:10FC4000AF51AE5012FC8A0551E55170020550C308
:10FC5000E55094F440E1D2AF75840075EF0122C203
:10FC6000AF75840F53A1FEE4F5B1F58443B701F5F8
:10FC700084438F018E088F098F828E83EDF0E4F527
:10FC800084538FFEF58453B7FE22C2AF75840F53A1
:10FC9000A1FE75B110E4F58443B701F584438F01EB
:10FCA0008E088F098F828E83EDF0E4F584538FFEEA
:10FCB000F58453B7FE22C2AF75B1218E0A8F0B8F28
:10FCC000828E83E493FF22C2AF75B1318E0A8F0B0F
:10FCD0008F828E83E493FF22C2AFE4FFFEE4F5B18E
:10FCE000F58443B701F584758F03AD07AC068C0826
:10FCF0008D098D828C83F0F58FF58453B7FE2FFF2D
:10FD000074043EFEC3948040D4E4F58453B7FE22CD
:10FD1000C2AF7F007E8075B110E4F58443B701F572
:04FD200084758F0354
:10FD2400AD07AC068C088D098D828C83F0F58FF5B8
:10FD34008453B7FE2FFF74043EFEC3648094744062
:08FD4400D1E4F58453B7FE225F
:0300000002007685
:0C007600787FE4F6D8FD7581A202627468
:10849200BB010689828A83E0225002E722BBFE02E8
:0984A200E32289828A83E493221B
:1084AB00BB010CE58229F582E5833AF583E0225086
:1084BB0006E92582F8E622BBFE06E92582F8E222D0
:0D84CB00E58229F582E5833AF583E49322EA
:1084D800BB010689828A83F0225002F722BBFE0183
:0284E800F3227D
:1084EA00EF8DF0A4A8F0CF8CF0A428CE8DF0A42EA6
:0284FA00FE2260
:1084FC00A3F8E0C5F025F0F0E58215827002158333
:06850C00E0C838F0E8228F
:10851200D083D082F8E4937012740193700DA3A3F8
:1085220093F8740193F5828883E47374029368600C
:06853200EFA3A3A380DF0C
:00000001FF
